Product: MDK-ARM Professional 5.10
Component: ARM Compiler 5.04 update 1 (build 49)
Tool: armlink [5040049]

==============================================================================

Section Cross References

    startup_stm32f10x_md.o(STACK) refers (Special) to heapauxi.o(.text) for __use_two_region_memory
    startup_stm32f10x_md.o(HEAP) refers (Special) to heapauxi.o(.text) for __use_two_region_memory
    startup_stm32f10x_md.o(RESET) refers (Special) to heapauxi.o(.text) for __use_two_region_memory
    startup_stm32f10x_md.o(RESET) refers to startup_stm32f10x_md.o(STACK) for __initial_sp
    startup_stm32f10x_md.o(RESET) refers to startup_stm32f10x_md.o(.text) for Reset_Handler
    startup_stm32f10x_md.o(RESET) refers to encoder.o(.text) for EXTI0_IRQHandler
    startup_stm32f10x_md.o(RESET) refers to exti.o(.text) for EXTI9_5_IRQHandler
    startup_stm32f10x_md.o(RESET) refers to control.o(.text) for TIM2_IRQHandler
    startup_stm32f10x_md.o(RESET) refers to usart3.o(.text) for USART3_IRQHandler
    startup_stm32f10x_md.o(.text) refers (Special) to heapauxi.o(.text) for __use_two_region_memory
    startup_stm32f10x_md.o(.text) refers to __main.o(!!!main) for __main
    startup_stm32f10x_md.o(.text) refers to startup_stm32f10x_md.o(HEAP) for Heap_Mem
    startup_stm32f10x_md.o(.text) refers to startup_stm32f10x_md.o(STACK) for Stack_Mem
    minibalance.o(.text) refers to sys.o(.text) for Stm32_Clock_Init
    minibalance.o(.text) refers to delay.o(.text) for delay_init
    minibalance.o(.text) refers to led.o(.text) for LED_Init
    minibalance.o(.text) refers to key.o(.text) for KEY_Init
    minibalance.o(.text) refers to oled.o(.text) for OLED_Init
    minibalance.o(.text) refers to encoder.o(.text) for Encoder_Init_TIM2
    minibalance.o(.text) refers to exti.o(.text) for EXTI_Init
    minibalance.o(.text) refers to motor.o(.text) for Servo_PWM_Init
    minibalance.o(.text) refers to usart.o(.text) for uart_init
    minibalance.o(.text) refers to adc.o(.text) for Adc_Init
    minibalance.o(.text) refers to usart3.o(.text) for uart3_init
    minibalance.o(.text) refers to pstwo.o(.text) for PS2_Init
    minibalance.o(.text) refers to stmflash.o(.text) for Flash_Read
    minibalance.o(.text) refers to timer.o(.text) for Timer_Init
    minibalance.o(.text) refers to show.o(.text) for APP_Show
    minibalance.o(.text) refers to minibalance.o(.data) for Flag_Way
    delay.o(.text) refers to delay.o(.data) for fac_us
    sys.o(.text) refers to sys.o(.emb_text) for WFI_SET
    usart.o(.text) refers (Special) to use_no_semi_2.o(.text) for __use_no_semihosting
    usart.o(.text) refers to fflt_clz.o(x$fpl$ffltu) for __aeabi_ui2f
    usart.o(.text) refers to fdiv.o(x$fpl$fdiv) for __aeabi_fdiv
    usart.o(.text) refers to ffixu.o(x$fpl$ffixu) for __aeabi_f2uiz
    usart.o(.text) refers to faddsub_clz.o(x$fpl$frsb) for __aeabi_frsub
    usart.o(.text) refers to fmul.o(x$fpl$fmul) for __aeabi_fmul
    usart.o(.text) refers to minibalance.o(.data) for Flag_Show
    usart.o(.data) refers (Special) to use_no_semi_2.o(.text) for __use_no_semihosting
    led.o(.text) refers to led.o(.data) for temp
    key.o(.text) refers to show.o(.text) for oled_show_once
    key.o(.text) refers to oled.o(.text) for OLED_Clear
    key.o(.text) refers to key.o(.data) for Forever_count
    key.o(.text) refers to minibalance.o(.data) for Encoder_Temp
    oled.o(.text) refers to delay.o(.text) for delay_ms
    oled.o(.text) refers to oled.o(.bss) for OLED_GRAM
    oled.o(.text) refers to oled.o(.constdata) for oled_asc2_1206
    adc.o(.text) refers to dflt_clz.o(x$fpl$dfltu) for __aeabi_ui2d
    adc.o(.text) refers to dmul.o(x$fpl$dmul) for __aeabi_dmul
    adc.o(.text) refers to ddiv.o(x$fpl$ddiv) for __aeabi_ddiv
    adc.o(.text) refers to dfix.o(x$fpl$dfix) for __aeabi_d2iz
    adc.o(.text) refers to usart.o(.text) for usart1_send
    adc.o(.text) refers to delay.o(.text) for delay_ms
    adc.o(.text) refers to minibalance.o(.bss) for ADV
    timer.o(.text) refers to sys.o(.text) for MY_NVIC_Init
    encoder.o(.text) refers to sys.o(.text) for Ex_NVIC_Config
    encoder.o(.text) refers to minibalance.o(.data) for Encoder_A_EXTI
    usart3.o(.text) refers to fflt_clz.o(x$fpl$ffltu) for __aeabi_ui2f
    usart3.o(.text) refers to fdiv.o(x$fpl$fdiv) for __aeabi_fdiv
    usart3.o(.text) refers to ffixu.o(x$fpl$ffixu) for __aeabi_f2uiz
    usart3.o(.text) refers to faddsub_clz.o(x$fpl$frsb) for __aeabi_frsub
    usart3.o(.text) refers to fmul.o(x$fpl$fmul) for __aeabi_fmul
    usart3.o(.text) refers to sys.o(.text) for MY_NVIC_Init
    usart3.o(.text) refers to dflt_clz.o(x$fpl$dflt) for __aeabi_i2d
    usart3.o(.text) refers to pow.o(i.pow) for pow
    usart3.o(.text) refers to dmul.o(x$fpl$dmul) for __aeabi_dmul
    usart3.o(.text) refers to f2d.o(x$fpl$f2d) for __aeabi_f2d
    usart3.o(.text) refers to daddsub_clz.o(x$fpl$dadd) for __aeabi_dadd
    usart3.o(.text) refers to d2f.o(x$fpl$d2f) for __aeabi_d2f
    usart3.o(.text) refers to rt_memclr.o(.text) for __aeabi_memclr
    usart3.o(.text) refers to usart3.o(.data) for Usart3_Receive
    usart3.o(.text) refers to minibalance.o(.data) for APP_RX
    usart3.o(.text) refers to usart3.o(.bss) for Receive
    pstwo.o(.text) refers to delay.o(.text) for delay_us
    pstwo.o(.text) refers to pstwo.o(.bss) for Data
    pstwo.o(.text) refers to pstwo.o(.data) for Comd
    exti.o(.text) refers to sys.o(.text) for Ex_NVIC_Config
    exti.o(.text) refers to minibalance.o(.data) for Flag_Next
    stmflash.o(.text) refers to delay.o(.text) for delay_us
    stmflash.o(.text) refers to fflt_clz.o(x$fpl$ffltu) for __aeabi_ui2f
    stmflash.o(.text) refers to ffixu.o(x$fpl$ffixu) for __aeabi_f2uiz
    stmflash.o(.text) refers to stmflash.o(.bss) for STMFLASH_BUF
    stmflash.o(.text) refers to minibalance.o(.bss) for PID_Parameter
    stmflash.o(.text) refers to minibalance.o(.data) for Bluetooth_Velocity
    control.o(.text) refers to f2d.o(x$fpl$f2d) for __aeabi_f2d
    control.o(.text) refers to tan.o(i.tan) for tan
    control.o(.text) refers to dmul.o(x$fpl$dmul) for __aeabi_dmul
    control.o(.text) refers to ddiv.o(x$fpl$ddiv) for __aeabi_ddiv
    control.o(.text) refers to daddsub_clz.o(x$fpl$dadd) for __aeabi_dadd
    control.o(.text) refers to dfix.o(x$fpl$dfix) for __aeabi_d2iz
    control.o(.text) refers to daddsub_clz.o(x$fpl$drsb) for __aeabi_drsub
    control.o(.text) refers to fmul.o(x$fpl$fmul) for __aeabi_fmul
    control.o(.text) refers to faddsub_clz.o(x$fpl$fadd) for __aeabi_fadd
    control.o(.text) refers to ffix.o(x$fpl$ffix) for __aeabi_f2iz
    control.o(.text) refers to fflt_clz.o(x$fpl$fflt) for __aeabi_i2f
    control.o(.text) refers to fflt_clz.o(x$fpl$ffltu) for __aeabi_ui2f
    control.o(.text) refers to fleqf.o(x$fpl$fleqf) for __aeabi_cfcmple
    control.o(.text) refers to frleqf.o(x$fpl$frleqf) for __aeabi_cfrcmple
    control.o(.text) refers to minibalance.o(.data) for Target_A
    control.o(.text) refers to control.o(.data) for Bias
    control.o(.text) refers to fdiv.o(x$fpl$fdiv) for __aeabi_fdiv
    control.o(.text) refers to faddsub_clz.o(x$fpl$fsub) for __aeabi_fsub
    control.o(.text) refers to d2f.o(x$fpl$d2f) for __aeabi_d2f
    control.o(.text) refers to key.o(.text) for click
    control.o(.text) refers to adc.o(.text) for RD_TSL
    control.o(.text) refers to minibalance.o(.bss) for ADV
    control.o(.text) refers to encoder.o(.text) for Read_Encoder
    control.o(.text) refers to led.o(.text) for Led_Flash
    show.o(.text) refers to _printf_percent.o(.ARM.Collect$$_printf_percent$$00000000) for _printf_percent
    show.o(.text) refers to _printf_d.o(.ARM.Collect$$_printf_percent$$00000009) for _printf_d
    show.o(.text) refers to _printf_dec.o(.text) for _printf_int_dec
    show.o(.text) refers to oled.o(.text) for OLED_DrawPoint
    show.o(.text) refers to dflt_clz.o(x$fpl$dflt) for __aeabi_i2d
    show.o(.text) refers to dmul.o(x$fpl$dmul) for __aeabi_dmul
    show.o(.text) refers to dfix.o(x$fpl$dfix) for __aeabi_d2iz
    show.o(.text) refers to ffix.o(x$fpl$ffix) for __aeabi_f2iz
    show.o(.text) refers to minibalance.o(.bss) for ADV
    show.o(.text) refers to minibalance.o(.data) for CCD_Yuzhi
    show.o(.text) refers to show.o(.data) for flag
    show.o(.text) refers to noretval__2printf.o(.text) for __2printf
    show.o(.text) refers to fflt_clz.o(x$fpl$fflt) for __aeabi_i2f
    show.o(.text) refers to datascope_dp.o(.text) for DataScope_Get_Channel_Data
    show.o(.text) refers to datascope_dp.o(.bss) for DataScope_OutPut_Buffer
    datascope_dp.o(.text) refers to datascope_dp.o(.bss) for DataScope_OutPut_Buffer
    use_no_semi_2.o(.text) refers (Special) to use_no_semi.o(.text) for __use_no_semihosting_swi
    __2printf.o(.text) refers to _printf_char_file.o(.text) for _printf_char_file
    __2printf.o(.text) refers to usart.o(.data) for __stdout
    noretval__2printf.o(.text) refers to _printf_char_file.o(.text) for _printf_char_file
    noretval__2printf.o(.text) refers to usart.o(.data) for __stdout
    __printf.o(.text) refers to _printf_percent.o(.ARM.Collect$$_printf_percent$$00000000) for _printf_percent
    _printf_dec.o(.text) refers to _printf_intcommon.o(.text) for _printf_int_common
    __printf_flags.o(.text) refers to _printf_percent.o(.ARM.Collect$$_printf_percent$$00000000) for _printf_percent
    __printf_flags.o(.text) refers to __printf_flags.o(.constdata) for .constdata
    __printf_ss.o(.text) refers to _printf_percent.o(.ARM.Collect$$_printf_percent$$00000000) for _printf_percent
    __printf_flags_ss.o(.text) refers to _printf_percent.o(.ARM.Collect$$_printf_percent$$00000000) for _printf_percent
    __printf_flags_ss.o(.text) refers to __printf_flags_ss.o(.constdata) for .constdata
    __printf_wp.o(.text) refers to __printf_wp.o(i._is_digit) for _is_digit
    __printf_wp.o(.text) refers to _printf_percent.o(.ARM.Collect$$_printf_percent$$00000000) for _printf_percent
    __printf_flags_wp.o(.text) refers to __printf_wp.o(i._is_digit) for _is_digit
    __printf_flags_wp.o(.text) refers to _printf_percent.o(.ARM.Collect$$_printf_percent$$00000000) for _printf_percent
    __printf_flags_wp.o(.text) refers to __printf_flags_wp.o(.constdata) for .constdata
    __printf_ss_wp.o(.text) refers to __printf_wp.o(i._is_digit) for _is_digit
    __printf_ss_wp.o(.text) refers to _printf_percent.o(.ARM.Collect$$_printf_percent$$00000000) for _printf_percent
    __printf_flags_ss_wp.o(.text) refers to __printf_wp.o(i._is_digit) for _is_digit
    __printf_flags_ss_wp.o(.text) refers to _printf_percent.o(.ARM.Collect$$_printf_percent$$00000000) for _printf_percent
    __printf_flags_ss_wp.o(.text) refers to __printf_flags_ss_wp.o(.constdata) for .constdata
    _printf_d.o(.ARM.Collect$$_printf_percent$$00000009) refers (Weak) to _printf_dec.o(.text) for _printf_int_dec
    _printf_percent.o(.ARM.Collect$$_printf_percent$$00000000) refers (Special) to _printf_percent_end.o(.ARM.Collect$$_printf_percent$$00000017) for _printf_percent_end
    rt_memclr.o(.text) refers to rt_memclr_w.o(.text) for _memset_w
    __main.o(!!!main) refers to rtentry.o(.ARM.Collect$$rtentry$$00000000) for __rt_entry
    d2f.o(x$fpl$d2f) refers (Special) to usenofp.o(x$fpl$usenofp) for __I$use$fp
    d2f.o(x$fpl$d2f) refers to fretinf.o(x$fpl$fretinf) for __fpl_fretinf
    d2f.o(x$fpl$d2f) refers to dnaninf.o(x$fpl$dnaninf) for __fpl_dnaninf
    daddsub_clz.o(x$fpl$dadd) refers (Special) to usenofp.o(x$fpl$usenofp) for __I$use$fp
    daddsub_clz.o(x$fpl$dadd) refers to daddsub_clz.o(x$fpl$dsub) for _dsub1
    daddsub_clz.o(x$fpl$dadd) refers to dretinf.o(x$fpl$dretinf) for __fpl_dretinf
    daddsub_clz.o(x$fpl$dadd) refers to dnaninf.o(x$fpl$dnaninf) for __fpl_dnaninf
    daddsub_clz.o(x$fpl$drsb) refers (Special) to usenofp.o(x$fpl$usenofp) for __I$use$fp
    daddsub_clz.o(x$fpl$drsb) refers to daddsub_clz.o(x$fpl$dadd) for _dadd1
    daddsub_clz.o(x$fpl$drsb) refers to daddsub_clz.o(x$fpl$dsub) for _dsub1
    daddsub_clz.o(x$fpl$dsub) refers (Special) to usenofp.o(x$fpl$usenofp) for __I$use$fp
    daddsub_clz.o(x$fpl$dsub) refers to daddsub_clz.o(x$fpl$dadd) for _dadd1
    daddsub_clz.o(x$fpl$dsub) refers to dnaninf.o(x$fpl$dnaninf) for __fpl_dnaninf
    ddiv.o(x$fpl$drdiv) refers (Special) to usenofp.o(x$fpl$usenofp) for __I$use$fp
    ddiv.o(x$fpl$drdiv) refers to ddiv.o(x$fpl$ddiv) for ddiv_entry
    ddiv.o(x$fpl$ddiv) refers (Special) to usenofp.o(x$fpl$usenofp) for __I$use$fp
    ddiv.o(x$fpl$ddiv) refers to dretinf.o(x$fpl$dretinf) for __fpl_dretinf
    ddiv.o(x$fpl$ddiv) refers to dnaninf.o(x$fpl$dnaninf) for __fpl_dnaninf
    dfix.o(x$fpl$dfix) refers (Special) to usenofp.o(x$fpl$usenofp) for __I$use$fp
    dfix.o(x$fpl$dfix) refers to dnaninf.o(x$fpl$dnaninf) for __fpl_dnaninf
    dfix.o(x$fpl$dfixr) refers (Special) to usenofp.o(x$fpl$usenofp) for __I$use$fp
    dfix.o(x$fpl$dfixr) refers to dnaninf.o(x$fpl$dnaninf) for __fpl_dnaninf
    dflt_clz.o(x$fpl$dfltu) refers (Special) to usenofp.o(x$fpl$usenofp) for __I$use$fp
    dflt_clz.o(x$fpl$dflt) refers (Special) to usenofp.o(x$fpl$usenofp) for __I$use$fp
    dflt_clz.o(x$fpl$dfltn) refers (Special) to usenofp.o(x$fpl$usenofp) for __I$use$fp
    dmul.o(x$fpl$dmul) refers (Special) to usenofp.o(x$fpl$usenofp) for __I$use$fp
    dmul.o(x$fpl$dmul) refers to dretinf.o(x$fpl$dretinf) for __fpl_dretinf
    dmul.o(x$fpl$dmul) refers to dnaninf.o(x$fpl$dnaninf) for __fpl_dnaninf
    f2d.o(x$fpl$f2d) refers (Special) to usenofp.o(x$fpl$usenofp) for __I$use$fp
    f2d.o(x$fpl$f2d) refers to fnaninf.o(x$fpl$fnaninf) for __fpl_fnaninf
    f2d.o(x$fpl$f2d) refers to dretinf.o(x$fpl$dretinf) for __fpl_dretinf
    faddsub_clz.o(x$fpl$fadd) refers (Special) to usenofp.o(x$fpl$usenofp) for __I$use$fp
    faddsub_clz.o(x$fpl$fadd) refers to faddsub_clz.o(x$fpl$fsub) for _fsub1
    faddsub_clz.o(x$fpl$fadd) refers to fretinf.o(x$fpl$fretinf) for __fpl_fretinf
    faddsub_clz.o(x$fpl$fadd) refers to fnaninf.o(x$fpl$fnaninf) for __fpl_fnaninf
    faddsub_clz.o(x$fpl$frsb) refers (Special) to usenofp.o(x$fpl$usenofp) for __I$use$fp
    faddsub_clz.o(x$fpl$frsb) refers to faddsub_clz.o(x$fpl$fadd) for _fadd1
    faddsub_clz.o(x$fpl$frsb) refers to faddsub_clz.o(x$fpl$fsub) for _fsub1
    faddsub_clz.o(x$fpl$fsub) refers (Special) to usenofp.o(x$fpl$usenofp) for __I$use$fp
    faddsub_clz.o(x$fpl$fsub) refers to faddsub_clz.o(x$fpl$fadd) for _fadd1
    faddsub_clz.o(x$fpl$fsub) refers to fnaninf.o(x$fpl$fnaninf) for __fpl_fnaninf
    fdiv.o(x$fpl$frdiv) refers (Special) to usenofp.o(x$fpl$usenofp) for __I$use$fp
    fdiv.o(x$fpl$frdiv) refers to fdiv.o(x$fpl$fdiv) for _fdiv1
    fdiv.o(x$fpl$fdiv) refers (Special) to usenofp.o(x$fpl$usenofp) for __I$use$fp
    fdiv.o(x$fpl$fdiv) refers to fretinf.o(x$fpl$fretinf) for __fpl_fretinf
    fdiv.o(x$fpl$fdiv) refers to fnaninf.o(x$fpl$fnaninf) for __fpl_fnaninf
    ffix.o(x$fpl$ffix) refers (Special) to usenofp.o(x$fpl$usenofp) for __I$use$fp
    ffix.o(x$fpl$ffix) refers to fnaninf.o(x$fpl$fnaninf) for __fpl_fnaninf
    ffix.o(x$fpl$ffixr) refers (Special) to usenofp.o(x$fpl$usenofp) for __I$use$fp
    ffix.o(x$fpl$ffixr) refers to fnaninf.o(x$fpl$fnaninf) for __fpl_fnaninf
    ffixu.o(x$fpl$ffixu) refers (Special) to usenofp.o(x$fpl$usenofp) for __I$use$fp
    ffixu.o(x$fpl$ffixu) refers to fnaninf.o(x$fpl$fnaninf) for __fpl_fnaninf
    ffixu.o(x$fpl$ffixur) refers (Special) to usenofp.o(x$fpl$usenofp) for __I$use$fp
    ffixu.o(x$fpl$ffixur) refers to fnaninf.o(x$fpl$fnaninf) for __fpl_fnaninf
    fflt_clz.o(x$fpl$ffltu) refers (Special) to usenofp.o(x$fpl$usenofp) for __I$use$fp
    fflt_clz.o(x$fpl$fflt) refers (Special) to usenofp.o(x$fpl$usenofp) for __I$use$fp
    fflt_clz.o(x$fpl$ffltn) refers (Special) to usenofp.o(x$fpl$usenofp) for __I$use$fp
    fleqf.o(x$fpl$fleqf) refers (Special) to usenofp.o(x$fpl$usenofp) for __I$use$fp
    fleqf.o(x$fpl$fleqf) refers to fnaninf.o(x$fpl$fnaninf) for __fpl_fnaninf
    fleqf.o(x$fpl$fleqf) refers to fcmpi.o(x$fpl$fcmpinf) for __fpl_fcmp_Inf
    fmul.o(x$fpl$fmul) refers (Special) to usenofp.o(x$fpl$usenofp) for __I$use$fp
    fmul.o(x$fpl$fmul) refers to fretinf.o(x$fpl$fretinf) for __fpl_fretinf
    fmul.o(x$fpl$fmul) refers to fnaninf.o(x$fpl$fnaninf) for __fpl_fnaninf
    frleqf.o(x$fpl$frleqf) refers (Special) to usenofp.o(x$fpl$usenofp) for __I$use$fp
    frleqf.o(x$fpl$frleqf) refers to fleqf.o(x$fpl$fleqf) for __fpl_fcmple_InfNaN
    pow.o(i.__softfp_pow) refers (Special) to usenofp.o(x$fpl$usenofp) for __I$use$fp
    pow.o(i.__softfp_pow) refers to pow.o(i.pow) for pow
    pow.o(i.pow) refers (Special) to usenofp.o(x$fpl$usenofp) for __I$use$fp
    pow.o(i.pow) refers to daddsub_clz.o(x$fpl$dadd) for __aeabi_dadd
    pow.o(i.pow) refers to _rserrno.o(.text) for __set_errno
    pow.o(i.pow) refers to ddiv.o(x$fpl$ddiv) for __aeabi_ddiv
    pow.o(i.pow) refers to sqrt.o(i.sqrt) for sqrt
    pow.o(i.pow) refers to dmul.o(x$fpl$dmul) for __aeabi_dmul
    pow.o(i.pow) refers to scalbn.o(x$fpl$scalbn) for __ARM_scalbn
    pow.o(i.pow) refers to dunder.o(i.__mathlib_dbl_underflow) for __mathlib_dbl_underflow
    pow.o(i.pow) refers to daddsub_clz.o(x$fpl$dsub) for __aeabi_dsub
    pow.o(i.pow) refers to daddsub_clz.o(x$fpl$drsb) for __aeabi_drsub
    pow.o(i.pow) refers to qnan.o(.constdata) for __mathlib_zero
    pow.o(i.pow) refers to poly.o(i.__kernel_poly) for __kernel_poly
    pow.o(i.pow) refers to dflt_clz.o(x$fpl$dflt) for __aeabi_i2d
    pow.o(i.pow) refers to drleqf.o(x$fpl$drleqf) for __aeabi_cdrcmple
    pow.o(i.pow) refers to pow.o(.constdata) for .constdata
    pow.o(i.pow) refers to fpclassify.o(i.__ARM_fpclassify) for __ARM_fpclassify
    pow.o(.constdata) refers (Special) to usenofp.o(x$fpl$usenofp) for __I$use$fp
    pow_x.o(i.____softfp_pow$lsc) refers (Special) to usenofp.o(x$fpl$usenofp) for __I$use$fp
    pow_x.o(i.____softfp_pow$lsc) refers to pow_x.o(i.__pow$lsc) for __pow$lsc
    pow_x.o(i.__pow$lsc) refers (Special) to usenofp.o(x$fpl$usenofp) for __I$use$fp
    pow_x.o(i.__pow$lsc) refers to daddsub_clz.o(x$fpl$dadd) for __aeabi_dadd
    pow_x.o(i.__pow$lsc) refers to _rserrno.o(.text) for __set_errno
    pow_x.o(i.__pow$lsc) refers to ddiv.o(x$fpl$ddiv) for __aeabi_ddiv
    pow_x.o(i.__pow$lsc) refers to sqrt.o(i.sqrt) for sqrt
    pow_x.o(i.__pow$lsc) refers to dmul.o(x$fpl$dmul) for __aeabi_dmul
    pow_x.o(i.__pow$lsc) refers to dflt_clz.o(x$fpl$dflt) for __aeabi_i2d
    pow_x.o(i.__pow$lsc) refers to daddsub_clz.o(x$fpl$dsub) for __aeabi_dsub
    pow_x.o(i.__pow$lsc) refers to scalbn.o(x$fpl$scalbn) for __ARM_scalbn
    pow_x.o(i.__pow$lsc) refers to daddsub_clz.o(x$fpl$drsb) for __aeabi_drsub
    pow_x.o(i.__pow$lsc) refers to qnan.o(.constdata) for __mathlib_zero
    pow_x.o(i.__pow$lsc) refers to pow_x.o(.constdata) for .constdata
    pow_x.o(i.__pow$lsc) refers to poly.o(i.__kernel_poly) for __kernel_poly
    pow_x.o(i.__pow$lsc) refers to drleqf.o(x$fpl$drleqf) for __aeabi_cdrcmple
    pow_x.o(.constdata) refers (Special) to usenofp.o(x$fpl$usenofp) for __I$use$fp
    tan.o(i.__softfp_tan) refers (Special) to usenofp.o(x$fpl$usenofp) for __I$use$fp
    tan.o(i.__softfp_tan) refers to _rserrno.o(.text) for __set_errno
    tan.o(i.__softfp_tan) refers to ddiv.o(x$fpl$ddiv) for __aeabi_ddiv
    tan.o(i.__softfp_tan) refers to scalbn.o(x$fpl$scalbn) for __ARM_scalbn
    tan.o(i.__softfp_tan) refers to rred.o(i.__ieee754_rem_pio2) for __ieee754_rem_pio2
    tan.o(i.__softfp_tan) refers to tan_i.o(i.__kernel_tan) for __kernel_tan
    tan.o(i.tan) refers (Special) to usenofp.o(x$fpl$usenofp) for __I$use$fp
    tan.o(i.tan) refers to _rserrno.o(.text) for __set_errno
    tan.o(i.tan) refers to ddiv.o(x$fpl$ddiv) for __aeabi_ddiv
    tan.o(i.tan) refers to scalbn.o(x$fpl$scalbn) for __ARM_scalbn
    tan.o(i.tan) refers to rred.o(i.__ieee754_rem_pio2) for __ieee754_rem_pio2
    tan.o(i.tan) refers to tan_i.o(i.__kernel_tan) for __kernel_tan
    tan_x.o(i.____softfp_tan$lsc) refers (Special) to usenofp.o(x$fpl$usenofp) for __I$use$fp
    tan_x.o(i.____softfp_tan$lsc) refers to _rserrno.o(.text) for __set_errno
    tan_x.o(i.____softfp_tan$lsc) refers to scalbn.o(x$fpl$scalbn) for __ARM_scalbn
    tan_x.o(i.____softfp_tan$lsc) refers to rred.o(i.__ieee754_rem_pio2) for __ieee754_rem_pio2
    tan_x.o(i.____softfp_tan$lsc) refers to tan_i.o(i.__kernel_tan) for __kernel_tan
    tan_x.o(i.__tan$lsc) refers (Special) to usenofp.o(x$fpl$usenofp) for __I$use$fp
    tan_x.o(i.__tan$lsc) refers to _rserrno.o(.text) for __set_errno
    tan_x.o(i.__tan$lsc) refers to scalbn.o(x$fpl$scalbn) for __ARM_scalbn
    tan_x.o(i.__tan$lsc) refers to rred.o(i.__ieee754_rem_pio2) for __ieee754_rem_pio2
    tan_x.o(i.__tan$lsc) refers to tan_i.o(i.__kernel_tan) for __kernel_tan
    rtentry.o(.ARM.Collect$$rtentry$$00000000) refers (Special) to rtentry2.o(.ARM.Collect$$rtentry$$0000000A) for __rt_entry_li
    rtentry.o(.ARM.Collect$$rtentry$$00000000) refers (Special) to rtentry2.o(.ARM.Collect$$rtentry$$0000000D) for __rt_entry_main
    rtentry.o(.ARM.Collect$$rtentry$$00000000) refers (Special) to rtentry2.o(.ARM.Collect$$rtentry$$0000000C) for __rt_entry_postli_1
    rtentry.o(.ARM.Collect$$rtentry$$00000000) refers (Special) to rtentry2.o(.ARM.Collect$$rtentry$$00000009) for __rt_entry_postsh_1
    rtentry.o(.ARM.Collect$$rtentry$$00000000) refers (Special) to rtentry2.o(.ARM.Collect$$rtentry$$00000002) for __rt_entry_presh_1
    rtentry.o(.ARM.Collect$$rtentry$$00000000) refers (Special) to rtentry4.o(.ARM.Collect$$rtentry$$00000004) for __rt_entry_sh
    _rserrno.o(.text) refers to rt_errno_addr_intlibspace.o(.text) for __aeabi_errno_addr
    _printf_char_file.o(.text) refers to _printf_char_common.o(.text) for _printf_char_common
    _printf_char_file.o(.text) refers to ferror.o(.text) for ferror
    _printf_char_file.o(.text) refers to usart.o(.text) for fputc
    dnaninf.o(x$fpl$dnaninf) refers (Special) to usenofp.o(x$fpl$usenofp) for __I$use$fp
    dretinf.o(x$fpl$dretinf) refers (Special) to usenofp.o(x$fpl$usenofp) for __I$use$fp
    drleqf.o(x$fpl$drleqf) refers (Special) to usenofp.o(x$fpl$usenofp) for __I$use$fp
    drleqf.o(x$fpl$drleqf) refers to dleqf.o(x$fpl$dleqf) for __fpl_dcmple_InfNaN
    fcmpi.o(x$fpl$fcmpinf) refers (Special) to usenofp.o(x$fpl$usenofp) for __I$use$fp
    fnaninf.o(x$fpl$fnaninf) refers (Special) to usenofp.o(x$fpl$usenofp) for __I$use$fp
    fretinf.o(x$fpl$fretinf) refers (Special) to usenofp.o(x$fpl$usenofp) for __I$use$fp
    scalbn.o(x$fpl$scalbn) refers (Special) to usenofp.o(x$fpl$usenofp) for __I$use$fp
    scalbn.o(x$fpl$scalbn) refers to dcheck1.o(x$fpl$dcheck1) for __fpl_dcheck_NaN1
    dunder.o(i.__mathlib_dbl_underflow) refers to scalbn.o(x$fpl$scalbn) for __ARM_scalbn
    fpclassify.o(i.__ARM_fpclassify) refers (Special) to usenofp.o(x$fpl$usenofp) for __I$use$fp
    poly.o(i.__kernel_poly) refers (Special) to usenofp.o(x$fpl$usenofp) for __I$use$fp
    poly.o(i.__kernel_poly) refers to dmul.o(x$fpl$dmul) for __aeabi_dmul
    poly.o(i.__kernel_poly) refers to daddsub_clz.o(x$fpl$dadd) for __aeabi_dadd
    qnan.o(.constdata) refers (Special) to usenofp.o(x$fpl$usenofp) for __I$use$fp
    rred.o(i.__ieee754_rem_pio2) refers (Special) to usenofp.o(x$fpl$usenofp) for __I$use$fp
    rred.o(i.__ieee754_rem_pio2) refers to daddsub_clz.o(x$fpl$dsub) for __aeabi_dsub
    rred.o(i.__ieee754_rem_pio2) refers to daddsub_clz.o(x$fpl$dadd) for __aeabi_dadd
    rred.o(i.__ieee754_rem_pio2) refers to dmul.o(x$fpl$dmul) for __aeabi_dmul
    rred.o(i.__ieee754_rem_pio2) refers to dfix.o(x$fpl$dfix) for __aeabi_d2iz
    rred.o(i.__ieee754_rem_pio2) refers to dflt_clz.o(x$fpl$dflt) for __aeabi_i2d
    rred.o(i.__ieee754_rem_pio2) refers to daddsub_clz.o(x$fpl$drsb) for __aeabi_drsub
    rred.o(i.__ieee754_rem_pio2) refers to dflt_clz.o(x$fpl$dfltu) for __aeabi_ui2d
    rred.o(i.__ieee754_rem_pio2) refers to scalbn.o(x$fpl$scalbn) for __ARM_scalbn
    rred.o(i.__ieee754_rem_pio2) refers to rred.o(.constdata) for .constdata
    rred.o(i.__use_accurate_range_reduction) refers (Special) to usenofp.o(x$fpl$usenofp) for __I$use$fp
    rred.o(.constdata) refers (Special) to usenofp.o(x$fpl$usenofp) for __I$use$fp
    sqrt.o(i.__softfp_sqrt) refers (Special) to usenofp.o(x$fpl$usenofp) for __I$use$fp
    sqrt.o(i.__softfp_sqrt) refers to dsqrt_noumaal.o(x$fpl$dsqrt) for _dsqrt
    sqrt.o(i.__softfp_sqrt) refers to _rserrno.o(.text) for __set_errno
    sqrt.o(i.sqrt) refers (Special) to usenofp.o(x$fpl$usenofp) for __I$use$fp
    sqrt.o(i.sqrt) refers to dsqrt_noumaal.o(x$fpl$dsqrt) for _dsqrt
    sqrt.o(i.sqrt) refers to _rserrno.o(.text) for __set_errno
    sqrt_x.o(i.____softfp_sqrt$lsc) refers (Special) to usenofp.o(x$fpl$usenofp) for __I$use$fp
    sqrt_x.o(i.____softfp_sqrt$lsc) refers to dleqf.o(x$fpl$dleqf) for __aeabi_cdcmple
    sqrt_x.o(i.____softfp_sqrt$lsc) refers to _rserrno.o(.text) for __set_errno
    sqrt_x.o(i.____softfp_sqrt$lsc) refers to dsqrt_noumaal.o(x$fpl$dsqrt) for _dsqrt
    sqrt_x.o(i.__sqrt$lsc) refers (Special) to usenofp.o(x$fpl$usenofp) for __I$use$fp
    sqrt_x.o(i.__sqrt$lsc) refers to dleqf.o(x$fpl$dleqf) for __aeabi_cdcmple
    sqrt_x.o(i.__sqrt$lsc) refers to _rserrno.o(.text) for __set_errno
    sqrt_x.o(i.__sqrt$lsc) refers to dsqrt_noumaal.o(x$fpl$dsqrt) for _dsqrt
    tan_i.o(i.__kernel_tan) refers (Special) to usenofp.o(x$fpl$usenofp) for __I$use$fp
    tan_i.o(i.__kernel_tan) refers to dfix.o(x$fpl$dfix) for __aeabi_d2iz
    tan_i.o(i.__kernel_tan) refers to daddsub_clz.o(x$fpl$drsb) for __aeabi_drsub
    tan_i.o(i.__kernel_tan) refers to daddsub_clz.o(x$fpl$dsub) for __aeabi_dsub
    tan_i.o(i.__kernel_tan) refers to daddsub_clz.o(x$fpl$dadd) for __aeabi_dadd
    tan_i.o(i.__kernel_tan) refers to dmul.o(x$fpl$dmul) for __aeabi_dmul
    tan_i.o(i.__kernel_tan) refers to poly.o(i.__kernel_poly) for __kernel_poly
    tan_i.o(i.__kernel_tan) refers to dflt_clz.o(x$fpl$dflt) for __aeabi_i2d
    tan_i.o(i.__kernel_tan) refers to ddiv.o(x$fpl$ddiv) for __aeabi_ddiv
    tan_i.o(i.__kernel_tan) refers to scalbn.o(x$fpl$scalbn) for __ARM_scalbn
    tan_i.o(i.__kernel_tan) refers to fpclassify.o(i.__ARM_fpclassify) for __ARM_fpclassify
    tan_i.o(i.__kernel_tan) refers to dunder.o(i.__mathlib_dbl_underflow) for __mathlib_dbl_underflow
    tan_i.o(i.__kernel_tan) refers to tan_i.o(.constdata) for .constdata
    tan_i.o(.constdata) refers (Special) to usenofp.o(x$fpl$usenofp) for __I$use$fp
    tan_i_x.o(i.____kernel_tan$lsc) refers (Special) to usenofp.o(x$fpl$usenofp) for __I$use$fp
    tan_i_x.o(i.____kernel_tan$lsc) refers to dfix.o(x$fpl$dfix) for __aeabi_d2iz
    tan_i_x.o(i.____kernel_tan$lsc) refers to daddsub_clz.o(x$fpl$drsb) for __aeabi_drsub
    tan_i_x.o(i.____kernel_tan$lsc) refers to daddsub_clz.o(x$fpl$dsub) for __aeabi_dsub
    tan_i_x.o(i.____kernel_tan$lsc) refers to daddsub_clz.o(x$fpl$dadd) for __aeabi_dadd
    tan_i_x.o(i.____kernel_tan$lsc) refers to dmul.o(x$fpl$dmul) for __aeabi_dmul
    tan_i_x.o(i.____kernel_tan$lsc) refers to poly.o(i.__kernel_poly) for __kernel_poly
    tan_i_x.o(i.____kernel_tan$lsc) refers to dflt_clz.o(x$fpl$dflt) for __aeabi_i2d
    tan_i_x.o(i.____kernel_tan$lsc) refers to ddiv.o(x$fpl$ddiv) for __aeabi_ddiv
    tan_i_x.o(i.____kernel_tan$lsc) refers to scalbn.o(x$fpl$scalbn) for __ARM_scalbn
    tan_i_x.o(i.____kernel_tan$lsc) refers to tan_i_x.o(.constdata) for .constdata
    tan_i_x.o(.constdata) refers (Special) to usenofp.o(x$fpl$usenofp) for __I$use$fp
    rtentry2.o(.ARM.Collect$$rtentry$$00000008) refers to boardinit2.o(.text) for _platform_post_stackheap_init
    rtentry2.o(.ARM.Collect$$rtentry$$0000000A) refers to libinit.o(.ARM.Collect$$libinit$$00000000) for __rt_lib_init
    rtentry2.o(.ARM.Collect$$rtentry$$0000000B) refers to boardinit3.o(.text) for _platform_post_lib_init
    rtentry2.o(.ARM.Collect$$rtentry$$0000000D) refers to minibalance.o(.text) for main
    rtentry2.o(.ARM.Collect$$rtentry$$0000000D) refers to exit.o(.text) for exit
    rtentry2.o(.ARM.exidx) refers to rtentry2.o(.ARM.Collect$$rtentry$$00000001) for .ARM.Collect$$rtentry$$00000001
    rtentry2.o(.ARM.exidx) refers to rtentry2.o(.ARM.Collect$$rtentry$$00000008) for .ARM.Collect$$rtentry$$00000008
    rtentry2.o(.ARM.exidx) refers to rtentry2.o(.ARM.Collect$$rtentry$$0000000A) for .ARM.Collect$$rtentry$$0000000A
    rtentry2.o(.ARM.exidx) refers to rtentry2.o(.ARM.Collect$$rtentry$$0000000B) for .ARM.Collect$$rtentry$$0000000B
    rtentry2.o(.ARM.exidx) refers to rtentry2.o(.ARM.Collect$$rtentry$$0000000D) for .ARM.Collect$$rtentry$$0000000D
    rtentry4.o(.ARM.Collect$$rtentry$$00000004) refers to sys_stackheap_outer.o(.text) for __user_setup_stackheap
    rtentry4.o(.ARM.exidx) refers to rtentry4.o(.ARM.Collect$$rtentry$$00000004) for .ARM.Collect$$rtentry$$00000004
    rt_errno_addr.o(.text) refers to rt_errno_addr.o(.bss) for __aeabi_errno_addr_data
    rt_errno_addr_intlibspace.o(.text) refers to libspace.o(.bss) for __libspace_start
    _printf_char_common.o(.text) refers to __printf.o(.text) for __printf
    dcheck1.o(x$fpl$dcheck1) refers (Special) to usenofp.o(x$fpl$usenofp) for __I$use$fp
    dcheck1.o(x$fpl$dcheck1) refers to retnan.o(x$fpl$retnan) for __fpl_return_NaN
    dleqf.o(x$fpl$dleqf) refers (Special) to usenofp.o(x$fpl$usenofp) for __I$use$fp
    dleqf.o(x$fpl$dleqf) refers to dnaninf.o(x$fpl$dnaninf) for __fpl_dnaninf
    dleqf.o(x$fpl$dleqf) refers to dcmpi.o(x$fpl$dcmpinf) for __fpl_dcmp_Inf
    dsqrt_noumaal.o(x$fpl$dsqrt) refers (Special) to usenofp.o(x$fpl$usenofp) for __I$use$fp
    dsqrt_noumaal.o(x$fpl$dsqrt) refers to dnaninf.o(x$fpl$dnaninf) for __fpl_dnaninf
    libspace.o(.text) refers to libspace.o(.bss) for __libspace_start
    sys_stackheap_outer.o(.text) refers to libspace.o(.text) for __user_perproc_libspace
    sys_stackheap_outer.o(.text) refers to startup_stm32f10x_md.o(.text) for __user_initial_stackheap
    exit.o(.text) refers to rtexit.o(.ARM.Collect$$rtexit$$00000000) for __rt_exit
    libinit.o(.ARM.Collect$$libinit$$00000000) refers (Special) to libinit2.o(.ARM.Collect$$libinit$$0000002C) for __rt_lib_init_alloca_1
    libinit.o(.ARM.Collect$$libinit$$00000000) refers (Special) to libinit2.o(.ARM.Collect$$libinit$$0000002A) for __rt_lib_init_argv_1
    libinit.o(.ARM.Collect$$libinit$$00000000) refers (Special) to libinit2.o(.ARM.Collect$$libinit$$00000019) for __rt_lib_init_atexit_1
    libinit.o(.ARM.Collect$$libinit$$00000000) refers (Special) to libinit2.o(.ARM.Collect$$libinit$$0000001F) for __rt_lib_init_clock_1
    libinit.o(.ARM.Collect$$libinit$$00000000) refers (Special) to libinit2.o(.ARM.Collect$$libinit$$00000030) for __rt_lib_init_cpp_1
    libinit.o(.ARM.Collect$$libinit$$00000000) refers (Special) to libinit2.o(.ARM.Collect$$libinit$$0000002E) for __rt_lib_init_exceptions_1
    libinit.o(.ARM.Collect$$libinit$$00000000) refers (Special) to libinit2.o(.ARM.Collect$$libinit$$00000002) for __rt_lib_init_fp_1
    libinit.o(.ARM.Collect$$libinit$$00000000) refers (Special) to libinit2.o(.ARM.Collect$$libinit$$0000001D) for __rt_lib_init_fp_trap_1
    libinit.o(.ARM.Collect$$libinit$$00000000) refers (Special) to libinit2.o(.ARM.Collect$$libinit$$00000021) for __rt_lib_init_getenv_1
    libinit.o(.ARM.Collect$$libinit$$00000000) refers (Special) to libinit2.o(.ARM.Collect$$libinit$$00000008) for __rt_lib_init_heap_1
    libinit.o(.ARM.Collect$$libinit$$00000000) refers (Special) to libinit2.o(.ARM.Collect$$libinit$$0000000F) for __rt_lib_init_lc_collate_1
    libinit.o(.ARM.Collect$$libinit$$00000000) refers (Special) to libinit2.o(.ARM.Collect$$libinit$$00000011) for __rt_lib_init_lc_ctype_1
    libinit.o(.ARM.Collect$$libinit$$00000000) refers (Special) to libinit2.o(.ARM.Collect$$libinit$$00000013) for __rt_lib_init_lc_monetary_1
    libinit.o(.ARM.Collect$$libinit$$00000000) refers (Special) to libinit2.o(.ARM.Collect$$libinit$$00000015) for __rt_lib_init_lc_numeric_1
    libinit.o(.ARM.Collect$$libinit$$00000000) refers (Special) to libinit2.o(.ARM.Collect$$libinit$$00000017) for __rt_lib_init_lc_time_1
    libinit.o(.ARM.Collect$$libinit$$00000000) refers (Special) to libinit2.o(.ARM.Collect$$libinit$$0000000C) for __rt_lib_init_rand_1
    libinit.o(.ARM.Collect$$libinit$$00000000) refers (Special) to libinit2.o(.ARM.Collect$$libinit$$00000031) for __rt_lib_init_return
    libinit.o(.ARM.Collect$$libinit$$00000000) refers (Special) to libinit2.o(.ARM.Collect$$libinit$$0000001B) for __rt_lib_init_signal_1
    libinit.o(.ARM.Collect$$libinit$$00000000) refers (Special) to libinit2.o(.ARM.Collect$$libinit$$00000023) for __rt_lib_init_stdio_1
    libinit.o(.ARM.Collect$$libinit$$00000000) refers (Special) to libinit2.o(.ARM.Collect$$libinit$$0000000A) for __rt_lib_init_user_alloc_1
    dcmpi.o(x$fpl$dcmpinf) refers (Special) to usenofp.o(x$fpl$usenofp) for __I$use$fp
    retnan.o(x$fpl$retnan) refers (Special) to usenofp.o(x$fpl$usenofp) for __I$use$fp
    retnan.o(x$fpl$retnan) refers to trapv.o(x$fpl$trapveneer) for __fpl_cmpreturn
    rtexit.o(.ARM.Collect$$rtexit$$00000000) refers (Special) to rtexit2.o(.ARM.Collect$$rtexit$$00000004) for __rt_exit_exit
    rtexit.o(.ARM.Collect$$rtexit$$00000000) refers (Special) to rtexit2.o(.ARM.Collect$$rtexit$$00000003) for __rt_exit_ls
    rtexit.o(.ARM.Collect$$rtexit$$00000000) refers (Special) to rtexit2.o(.ARM.Collect$$rtexit$$00000002) for __rt_exit_prels_1
    rtexit.o(.ARM.exidx) refers (Special) to rtexit2.o(.ARM.Collect$$rtexit$$00000004) for __rt_exit_exit
    rtexit.o(.ARM.exidx) refers (Special) to rtexit2.o(.ARM.Collect$$rtexit$$00000003) for __rt_exit_ls
    rtexit.o(.ARM.exidx) refers (Special) to rtexit2.o(.ARM.Collect$$rtexit$$00000002) for __rt_exit_prels_1
    rtexit.o(.ARM.exidx) refers to rtexit.o(.ARM.Collect$$rtexit$$00000000) for .ARM.Collect$$rtexit$$00000000
    libinit2.o(.ARM.Collect$$libinit$$0000000E) refers to libinit2.o(.ARM.Collect$$libinit$$0000000D) for .ARM.Collect$$libinit$$0000000D
    libinit2.o(.ARM.Collect$$libinit$$00000010) refers to libinit2.o(.ARM.Collect$$libinit$$0000000D) for .ARM.Collect$$libinit$$0000000D
    libinit2.o(.ARM.Collect$$libinit$$00000012) refers to libinit2.o(.ARM.Collect$$libinit$$0000000D) for .ARM.Collect$$libinit$$0000000D
    libinit2.o(.ARM.Collect$$libinit$$00000014) refers to libinit2.o(.ARM.Collect$$libinit$$0000000D) for .ARM.Collect$$libinit$$0000000D
    libinit2.o(.ARM.Collect$$libinit$$00000016) refers to libinit2.o(.ARM.Collect$$libinit$$0000000D) for .ARM.Collect$$libinit$$0000000D
    libinit2.o(.ARM.Collect$$libinit$$00000024) refers to argv_veneer.o(.emb_text) for __ARM_argv_veneer
    libinit2.o(.ARM.Collect$$libinit$$00000025) refers to argv_veneer.o(.emb_text) for __ARM_argv_veneer
    trapv.o(x$fpl$trapveneer) refers (Special) to usenofp.o(x$fpl$usenofp) for __I$use$fp
    rtexit2.o(.ARM.Collect$$rtexit$$00000003) refers to libshutdown.o(.ARM.Collect$$libshutdown$$00000000) for __rt_lib_shutdown
    rtexit2.o(.ARM.Collect$$rtexit$$00000004) refers to usart.o(.text) for _sys_exit
    rtexit2.o(.ARM.exidx) refers to rtexit2.o(.ARM.Collect$$rtexit$$00000001) for .ARM.Collect$$rtexit$$00000001
    rtexit2.o(.ARM.exidx) refers to rtexit2.o(.ARM.Collect$$rtexit$$00000003) for .ARM.Collect$$rtexit$$00000003
    rtexit2.o(.ARM.exidx) refers to rtexit2.o(.ARM.Collect$$rtexit$$00000004) for .ARM.Collect$$rtexit$$00000004
    argv_veneer.o(.emb_text) refers to no_argv.o(.text) for __ARM_get_argv
    _get_argv_nomalloc.o(.text) refers (Special) to hrguard.o(.text) for __heap_region$guard
    _get_argv_nomalloc.o(.text) refers to defsig_rtmem_outer.o(.text) for __rt_SIGRTMEM
    _get_argv_nomalloc.o(.text) refers to sys_command.o(.text) for _sys_command_string
    libshutdown.o(.ARM.Collect$$libshutdown$$00000000) refers (Special) to libshutdown2.o(.ARM.Collect$$libshutdown$$00000006) for __rt_lib_shutdown_fp_trap_1
    libshutdown.o(.ARM.Collect$$libshutdown$$00000000) refers (Special) to libshutdown2.o(.ARM.Collect$$libshutdown$$0000000E) for __rt_lib_shutdown_heap_1
    libshutdown.o(.ARM.Collect$$libshutdown$$00000000) refers (Special) to libshutdown2.o(.ARM.Collect$$libshutdown$$0000000F) for __rt_lib_shutdown_return
    libshutdown.o(.ARM.Collect$$libshutdown$$00000000) refers (Special) to libshutdown2.o(.ARM.Collect$$libshutdown$$00000009) for __rt_lib_shutdown_signal_1
    libshutdown.o(.ARM.Collect$$libshutdown$$00000000) refers (Special) to libshutdown2.o(.ARM.Collect$$libshutdown$$00000003) for __rt_lib_shutdown_stdio_1
    libshutdown.o(.ARM.Collect$$libshutdown$$00000000) refers (Special) to libshutdown2.o(.ARM.Collect$$libshutdown$$0000000B) for __rt_lib_shutdown_user_alloc_1
    sys_command.o(.text) refers (Special) to use_no_semi.o(.text) for __I$use$semihosting
    sys_command.o(.text) refers (Special) to indicate_semi.o(.text) for __semihosting_library_function
    defsig_rtmem_outer.o(.text) refers to defsig_rtmem_inner.o(.text) for __rt_SIGRTMEM_inner
    defsig_rtmem_outer.o(.text) refers to defsig_exit.o(.text) for __sig_exit
    defsig_rtmem_formal.o(.text) refers to rt_raise.o(.text) for __rt_raise
    rt_raise.o(.text) refers to __raise.o(.text) for __raise
    rt_raise.o(.text) refers to usart.o(.text) for _sys_exit
    defsig_exit.o(.text) refers to usart.o(.text) for _sys_exit
    defsig_rtmem_inner.o(.text) refers to defsig_general.o(.text) for __default_signal_display
    __raise.o(.text) refers to defsig.o(CL$$defsig) for __default_signal_handler
    defsig_general.o(.text) refers to sys_wrch.o(.text) for _ttywrch
    sys_wrch.o(.text) refers (Special) to use_no_semi.o(.text) for __I$use$semihosting
    sys_wrch.o(.text) refers (Special) to indicate_semi.o(.text) for __semihosting_library_function
    defsig.o(CL$$defsig) refers to defsig_rtmem_inner.o(.text) for __rt_SIGRTMEM_inner
    defsig_abrt_inner.o(.text) refers to defsig_general.o(.text) for __default_signal_display
    defsig_fpe_inner.o(.text) refers to defsig_general.o(.text) for __default_signal_display
    defsig_rtred_inner.o(.text) refers to defsig_general.o(.text) for __default_signal_display
    defsig_stak_inner.o(.text) refers to defsig_general.o(.text) for __default_signal_display
    defsig_pvfn_inner.o(.text) refers to defsig_general.o(.text) for __default_signal_display
    defsig_cppl_inner.o(.text) refers to defsig_general.o(.text) for __default_signal_display
    defsig_segv_inner.o(.text) refers to defsig_general.o(.text) for __default_signal_display
    defsig_other.o(.text) refers to defsig_general.o(.text) for __default_signal_display


==============================================================================

Image Symbol Table

    Local Symbols

    Symbol Name                              Value     Ov Type        Size  Object(Section)

    ../clib/angel/boardlib.s                 0x00000000   Number         0  boardshut.o ABSOLUTE
    ../clib/angel/boardlib.s                 0x00000000   Number         0  boardinit3.o ABSOLUTE
    ../clib/angel/boardlib.s                 0x00000000   Number         0  boardinit2.o ABSOLUTE
    ../clib/angel/boardlib.s                 0x00000000   Number         0  boardinit1.o ABSOLUTE
    ../clib/angel/handlers.s                 0x00000000   Number         0  __scatter_copy.o ABSOLUTE
    ../clib/angel/handlers.s                 0x00000000   Number         0  __scatter_zi.o ABSOLUTE
    ../clib/angel/kernel.s                   0x00000000   Number         0  rtexit2.o ABSOLUTE
    ../clib/angel/kernel.s                   0x00000000   Number         0  rtentry.o ABSOLUTE
    ../clib/angel/kernel.s                   0x00000000   Number         0  rtentry2.o ABSOLUTE
    ../clib/angel/kernel.s                   0x00000000   Number         0  rtexit.o ABSOLUTE
    ../clib/angel/kernel.s                   0x00000000   Number         0  rtentry4.o ABSOLUTE
    ../clib/angel/rt.s                       0x00000000   Number         0  rt_errno_addr.o ABSOLUTE
    ../clib/angel/rt.s                       0x00000000   Number         0  rt_errno_addr_intlibspace.o ABSOLUTE
    ../clib/angel/rt.s                       0x00000000   Number         0  rt_raise.o ABSOLUTE
    ../clib/angel/scatter.s                  0x00000000   Number         0  __scatter.o ABSOLUTE
    ../clib/angel/startup.s                  0x00000000   Number         0  __main.o ABSOLUTE
    ../clib/angel/sys.s                      0x00000000   Number         0  sys_stackheap_outer.o ABSOLUTE
    ../clib/angel/sys.s                      0x00000000   Number         0  libspace.o ABSOLUTE
    ../clib/angel/sys.s                      0x00000000   Number         0  use_no_semi.o ABSOLUTE
    ../clib/angel/sys.s                      0x00000000   Number         0  use_no_semi_2.o ABSOLUTE
    ../clib/angel/sys.s                      0x00000000   Number         0  indicate_semi.o ABSOLUTE
    ../clib/angel/sysapp.c                   0x00000000   Number         0  sys_wrch.o ABSOLUTE
    ../clib/angel/sysapp.c                   0x00000000   Number         0  sys_command.o ABSOLUTE
    ../clib/armsys.c                         0x00000000   Number         0  _get_argv_nomalloc.o ABSOLUTE
    ../clib/armsys.c                         0x00000000   Number         0  argv_veneer.o ABSOLUTE
    ../clib/armsys.c                         0x00000000   Number         0  argv_veneer.o ABSOLUTE
    ../clib/armsys.c                         0x00000000   Number         0  no_argv.o ABSOLUTE
    ../clib/fenv.c                           0x00000000   Number         0  _rserrno.o ABSOLUTE
    ../clib/heapalloc.c                      0x00000000   Number         0  hrguard.o ABSOLUTE
    ../clib/heapaux.c                        0x00000000   Number         0  heapauxi.o ABSOLUTE
    ../clib/libinit.s                        0x00000000   Number         0  libinit.o ABSOLUTE
    ../clib/libinit.s                        0x00000000   Number         0  libshutdown2.o ABSOLUTE
    ../clib/libinit.s                        0x00000000   Number         0  libinit2.o ABSOLUTE
    ../clib/libinit.s                        0x00000000   Number         0  libshutdown.o ABSOLUTE
    ../clib/memcpset.s                       0x00000000   Number         0  rt_memclr_w.o ABSOLUTE
    ../clib/memcpset.s                       0x00000000   Number         0  rt_memclr.o ABSOLUTE
    ../clib/printf.c                         0x00000000   Number         0  __printf_nopercent.o ABSOLUTE
    ../clib/printf.c                         0x00000000   Number         0  __2printf.o ABSOLUTE
    ../clib/printf.c                         0x00000000   Number         0  __printf_ss.o ABSOLUTE
    ../clib/printf.c                         0x00000000   Number         0  noretval__2printf.o ABSOLUTE
    ../clib/printf.c                         0x00000000   Number         0  __printf.o ABSOLUTE
    ../clib/printf.c                         0x00000000   Number         0  _printf_dec.o ABSOLUTE
    ../clib/printf.c                         0x00000000   Number         0  _printf_char_common.o ABSOLUTE
    ../clib/printf.c                         0x00000000   Number         0  __printf_flags.o ABSOLUTE
    ../clib/printf.c                         0x00000000   Number         0  __printf_flags_ss.o ABSOLUTE
    ../clib/printf.c                         0x00000000   Number         0  __printf_wp.o ABSOLUTE
    ../clib/printf.c                         0x00000000   Number         0  __printf_flags_wp.o ABSOLUTE
    ../clib/printf.c                         0x00000000   Number         0  __printf_ss_wp.o ABSOLUTE
    ../clib/printf.c                         0x00000000   Number         0  __printf_flags_ss_wp.o ABSOLUTE
    ../clib/printf.c                         0x00000000   Number         0  _printf_char_file.o ABSOLUTE
    ../clib/printf.c                         0x00000000   Number         0  _printf_intcommon.o ABSOLUTE
    ../clib/printf_percent.s                 0x00000000   Number         0  _printf_d.o ABSOLUTE
    ../clib/printf_percent.s                 0x00000000   Number         0  _printf_percent_end.o ABSOLUTE
    ../clib/printf_percent.s                 0x00000000   Number         0  _printf_percent.o ABSOLUTE
    ../clib/signal.c                         0x00000000   Number         0  defsig_rtmem_formal.o ABSOLUTE
    ../clib/signal.c                         0x00000000   Number         0  defsig_rtmem_outer.o ABSOLUTE
    ../clib/signal.c                         0x00000000   Number         0  defsig_stak_inner.o ABSOLUTE
    ../clib/signal.c                         0x00000000   Number         0  defsig_exit.o ABSOLUTE
    ../clib/signal.c                         0x00000000   Number         0  defsig_rtmem_inner.o ABSOLUTE
    ../clib/signal.c                         0x00000000   Number         0  __raise.o ABSOLUTE
    ../clib/signal.c                         0x00000000   Number         0  defsig_other.o ABSOLUTE
    ../clib/signal.c                         0x00000000   Number         0  defsig_segv_inner.o ABSOLUTE
    ../clib/signal.c                         0x00000000   Number         0  defsig_cppl_inner.o ABSOLUTE
    ../clib/signal.c                         0x00000000   Number         0  defsig_pvfn_inner.o ABSOLUTE
    ../clib/signal.c                         0x00000000   Number         0  defsig_rtred_inner.o ABSOLUTE
    ../clib/signal.c                         0x00000000   Number         0  defsig_fpe_inner.o ABSOLUTE
    ../clib/signal.c                         0x00000000   Number         0  defsig_general.o ABSOLUTE
    ../clib/signal.c                         0x00000000   Number         0  defsig_abrt_inner.o ABSOLUTE
    ../clib/signal.s                         0x00000000   Number         0  defsig.o ABSOLUTE
    ../clib/stdio.c                          0x00000000   Number         0  ferror_locked.o ABSOLUTE
    ../clib/stdio.c                          0x00000000   Number         0  ferror.o ABSOLUTE
    ../clib/stdlib.c                         0x00000000   Number         0  exit.o ABSOLUTE
    ../fplib/d2f.s                           0x00000000   Number         0  d2f.o ABSOLUTE
    ../fplib/daddsub.s                       0x00000000   Number         0  daddsub_clz.o ABSOLUTE
    ../fplib/dcheck1.s                       0x00000000   Number         0  dcheck1.o ABSOLUTE
    ../fplib/dcmpi.s                         0x00000000   Number         0  dcmpi.o ABSOLUTE
    ../fplib/ddiv.s                          0x00000000   Number         0  ddiv.o ABSOLUTE
    ../fplib/dfix.s                          0x00000000   Number         0  dfix.o ABSOLUTE
    ../fplib/dflt.s                          0x00000000   Number         0  dflt_clz.o ABSOLUTE
    ../fplib/dleqf.s                         0x00000000   Number         0  dleqf.o ABSOLUTE
    ../fplib/dmul.s                          0x00000000   Number         0  dmul.o ABSOLUTE
    ../fplib/dnaninf.s                       0x00000000   Number         0  dnaninf.o ABSOLUTE
    ../fplib/dretinf.s                       0x00000000   Number         0  dretinf.o ABSOLUTE
    ../fplib/drleqf.s                        0x00000000   Number         0  drleqf.o ABSOLUTE
    ../fplib/dsqrt.s                         0x00000000   Number         0  dsqrt_noumaal.o ABSOLUTE
    ../fplib/f2d.s                           0x00000000   Number         0  f2d.o ABSOLUTE
    ../fplib/faddsub.s                       0x00000000   Number         0  faddsub_clz.o ABSOLUTE
    ../fplib/fcmpi.s                         0x00000000   Number         0  fcmpi.o ABSOLUTE
    ../fplib/fdiv.s                          0x00000000   Number         0  fdiv.o ABSOLUTE
    ../fplib/ffix.s                          0x00000000   Number         0  ffix.o ABSOLUTE
    ../fplib/ffixu.s                         0x00000000   Number         0  ffixu.o ABSOLUTE
    ../fplib/fflt.s                          0x00000000   Number         0  fflt_clz.o ABSOLUTE
    ../fplib/fleqf.s                         0x00000000   Number         0  fleqf.o ABSOLUTE
    ../fplib/fmul.s                          0x00000000   Number         0  fmul.o ABSOLUTE
    ../fplib/fnaninf.s                       0x00000000   Number         0  fnaninf.o ABSOLUTE
    ../fplib/fpinit.s                        0x00000000   Number         0  fpinit.o ABSOLUTE
    ../fplib/fretinf.s                       0x00000000   Number         0  fretinf.o ABSOLUTE
    ../fplib/frleqf.s                        0x00000000   Number         0  frleqf.o ABSOLUTE
    ../fplib/retnan.s                        0x00000000   Number         0  retnan.o ABSOLUTE
    ../fplib/scalbn.s                        0x00000000   Number         0  scalbn.o ABSOLUTE
    ../fplib/trapv.s                         0x00000000   Number         0  trapv.o ABSOLUTE
    ../fplib/usenofp.s                       0x00000000   Number         0  usenofp.o ABSOLUTE
    ../mathlib/dunder.c                      0x00000000   Number         0  dunder.o ABSOLUTE
    ../mathlib/fpclassify.c                  0x00000000   Number         0  fpclassify.o ABSOLUTE
    ../mathlib/poly.c                        0x00000000   Number         0  poly.o ABSOLUTE
    ../mathlib/pow.c                         0x00000000   Number         0  pow.o ABSOLUTE
    ../mathlib/pow.c                         0x00000000   Number         0  pow_x.o ABSOLUTE
    ../mathlib/qnan.c                        0x00000000   Number         0  qnan.o ABSOLUTE
    ../mathlib/rred.c                        0x00000000   Number         0  rred.o ABSOLUTE
    ../mathlib/sqrt.c                        0x00000000   Number         0  sqrt.o ABSOLUTE
    ../mathlib/sqrt.c                        0x00000000   Number         0  sqrt_x.o ABSOLUTE
    ../mathlib/tan.c                         0x00000000   Number         0  tan_x.o ABSOLUTE
    ../mathlib/tan.c                         0x00000000   Number         0  tan.o ABSOLUTE
    ../mathlib/tan_i.c                       0x00000000   Number         0  tan_i.o ABSOLUTE
    ../mathlib/tan_i.c                       0x00000000   Number         0  tan_i_x.o ABSOLUTE
    ..\BALANCE\CONTROL\control.c             0x00000000   Number         0  control.o ABSOLUTE
    ..\BALANCE\show\show.c                   0x00000000   Number         0  show.o ABSOLUTE
    ..\HARDWARE\ADC\adc.c                    0x00000000   Number         0  adc.o ABSOLUTE
    ..\HARDWARE\DataScope_DP\DataScope_DP.C  0x00000000   Number         0  datascope_dp.o ABSOLUTE
    ..\HARDWARE\ENCODER\encoder.c            0x00000000   Number         0  encoder.o ABSOLUTE
    ..\HARDWARE\EXTI\exti.c                  0x00000000   Number         0  exti.o ABSOLUTE
    ..\HARDWARE\KEY\key.c                    0x00000000   Number         0  key.o ABSOLUTE
    ..\HARDWARE\LED\LED.C                    0x00000000   Number         0  led.o ABSOLUTE
    ..\HARDWARE\MOTOR\motor.c                0x00000000   Number         0  motor.o ABSOLUTE
    ..\HARDWARE\OLED\oled.c                  0x00000000   Number         0  oled.o ABSOLUTE
    ..\HARDWARE\PS2\pstwo.c                  0x00000000   Number         0  pstwo.o ABSOLUTE
    ..\HARDWARE\STMFLASH\stmflash.c          0x00000000   Number         0  stmflash.o ABSOLUTE
    ..\HARDWARE\TIMER\timer.c                0x00000000   Number         0  timer.o ABSOLUTE
    ..\HARDWARE\USART3\usart3.c              0x00000000   Number         0  usart3.o ABSOLUTE
    ..\SYSTEM\delay\delay.c                  0x00000000   Number         0  delay.o ABSOLUTE
    ..\SYSTEM\sys\sys.c                      0x00000000   Number         0  sys.o ABSOLUTE
    ..\SYSTEM\usart\usart.c                  0x00000000   Number         0  usart.o ABSOLUTE
    ..\\SYSTEM\\sys\\sys.c                   0x00000000   Number         0  sys.o ABSOLUTE
    Minibalance.c                            0x00000000   Number         0  minibalance.o ABSOLUTE
    dc.s                                     0x00000000   Number         0  dc.o ABSOLUTE
    startup_stm32f10x_md.s                   0x00000000   Number         0  startup_stm32f10x_md.o ABSOLUTE
    RESET                                    0x08000000   Section      236  startup_stm32f10x_md.o(RESET)
    !!!main                                  0x080000ec   Section        8  __main.o(!!!main)
    !!!scatter                               0x080000f4   Section       52  __scatter.o(!!!scatter)
    !!handler_copy                           0x08000128   Section       26  __scatter_copy.o(!!handler_copy)
    !!handler_zi                             0x08000144   Section       28  __scatter_zi.o(!!handler_zi)
    .ARM.Collect$$_printf_percent$$00000000  0x08000160   Section        0  _printf_percent.o(.ARM.Collect$$_printf_percent$$00000000)
    .ARM.Collect$$_printf_percent$$00000009  0x08000160   Section        6  _printf_d.o(.ARM.Collect$$_printf_percent$$00000009)
    .ARM.Collect$$_printf_percent$$00000017  0x08000166   Section        4  _printf_percent_end.o(.ARM.Collect$$_printf_percent$$00000017)
    .ARM.Collect$$libinit$$00000000          0x0800016a   Section        2  libinit.o(.ARM.Collect$$libinit$$00000000)
    .ARM.Collect$$libinit$$00000002          0x0800016c   Section        0  libinit2.o(.ARM.Collect$$libinit$$00000002)
    .ARM.Collect$$libinit$$00000008          0x0800016c   Section        0  libinit2.o(.ARM.Collect$$libinit$$00000008)
    .ARM.Collect$$libinit$$0000000A          0x0800016c   Section        0  libinit2.o(.ARM.Collect$$libinit$$0000000A)
    .ARM.Collect$$libinit$$0000000C          0x0800016c   Section        0  libinit2.o(.ARM.Collect$$libinit$$0000000C)
    .ARM.Collect$$libinit$$0000000F          0x0800016c   Section        0  libinit2.o(.ARM.Collect$$libinit$$0000000F)
    .ARM.Collect$$libinit$$00000011          0x0800016c   Section        0  libinit2.o(.ARM.Collect$$libinit$$00000011)
    .ARM.Collect$$libinit$$00000013          0x0800016c   Section        0  libinit2.o(.ARM.Collect$$libinit$$00000013)
    .ARM.Collect$$libinit$$00000015          0x0800016c   Section        0  libinit2.o(.ARM.Collect$$libinit$$00000015)
    .ARM.Collect$$libinit$$00000017          0x0800016c   Section        0  libinit2.o(.ARM.Collect$$libinit$$00000017)
    .ARM.Collect$$libinit$$00000019          0x0800016c   Section        0  libinit2.o(.ARM.Collect$$libinit$$00000019)
    .ARM.Collect$$libinit$$0000001B          0x0800016c   Section        0  libinit2.o(.ARM.Collect$$libinit$$0000001B)
    .ARM.Collect$$libinit$$0000001D          0x0800016c   Section        0  libinit2.o(.ARM.Collect$$libinit$$0000001D)
    .ARM.Collect$$libinit$$0000001F          0x0800016c   Section        0  libinit2.o(.ARM.Collect$$libinit$$0000001F)
    .ARM.Collect$$libinit$$00000021          0x0800016c   Section        0  libinit2.o(.ARM.Collect$$libinit$$00000021)
    .ARM.Collect$$libinit$$00000023          0x0800016c   Section        0  libinit2.o(.ARM.Collect$$libinit$$00000023)
    .ARM.Collect$$libinit$$0000002A          0x0800016c   Section        0  libinit2.o(.ARM.Collect$$libinit$$0000002A)
    .ARM.Collect$$libinit$$0000002C          0x0800016c   Section        0  libinit2.o(.ARM.Collect$$libinit$$0000002C)
    .ARM.Collect$$libinit$$0000002E          0x0800016c   Section        0  libinit2.o(.ARM.Collect$$libinit$$0000002E)
    .ARM.Collect$$libinit$$00000030          0x0800016c   Section        0  libinit2.o(.ARM.Collect$$libinit$$00000030)
    .ARM.Collect$$libinit$$00000031          0x0800016c   Section        2  libinit2.o(.ARM.Collect$$libinit$$00000031)
    .ARM.Collect$$libshutdown$$00000000      0x0800016e   Section        2  libshutdown.o(.ARM.Collect$$libshutdown$$00000000)
    .ARM.Collect$$libshutdown$$00000003      0x08000170   Section        0  libshutdown2.o(.ARM.Collect$$libshutdown$$00000003)
    .ARM.Collect$$libshutdown$$00000006      0x08000170   Section        0  libshutdown2.o(.ARM.Collect$$libshutdown$$00000006)
    .ARM.Collect$$libshutdown$$00000009      0x08000170   Section        0  libshutdown2.o(.ARM.Collect$$libshutdown$$00000009)
    .ARM.Collect$$libshutdown$$0000000B      0x08000170   Section        0  libshutdown2.o(.ARM.Collect$$libshutdown$$0000000B)
    .ARM.Collect$$libshutdown$$0000000E      0x08000170   Section        0  libshutdown2.o(.ARM.Collect$$libshutdown$$0000000E)
    .ARM.Collect$$libshutdown$$0000000F      0x08000170   Section        2  libshutdown2.o(.ARM.Collect$$libshutdown$$0000000F)
    .ARM.Collect$$rtentry$$00000000          0x08000172   Section        0  rtentry.o(.ARM.Collect$$rtentry$$00000000)
    .ARM.Collect$$rtentry$$00000002          0x08000172   Section        0  rtentry2.o(.ARM.Collect$$rtentry$$00000002)
    .ARM.Collect$$rtentry$$00000004          0x08000172   Section        6  rtentry4.o(.ARM.Collect$$rtentry$$00000004)
    .ARM.Collect$$rtentry$$00000009          0x08000178   Section        0  rtentry2.o(.ARM.Collect$$rtentry$$00000009)
    .ARM.Collect$$rtentry$$0000000A          0x08000178   Section        4  rtentry2.o(.ARM.Collect$$rtentry$$0000000A)
    .ARM.Collect$$rtentry$$0000000C          0x0800017c   Section        0  rtentry2.o(.ARM.Collect$$rtentry$$0000000C)
    .ARM.Collect$$rtentry$$0000000D          0x0800017c   Section        8  rtentry2.o(.ARM.Collect$$rtentry$$0000000D)
    .ARM.Collect$$rtexit$$00000000           0x08000184   Section        2  rtexit.o(.ARM.Collect$$rtexit$$00000000)
    .ARM.Collect$$rtexit$$00000002           0x08000186   Section        0  rtexit2.o(.ARM.Collect$$rtexit$$00000002)
    .ARM.Collect$$rtexit$$00000003           0x08000186   Section        4  rtexit2.o(.ARM.Collect$$rtexit$$00000003)
    .ARM.Collect$$rtexit$$00000004           0x0800018a   Section        6  rtexit2.o(.ARM.Collect$$rtexit$$00000004)
    .emb_text                                0x08000190   Section       12  sys.o(.emb_text)
    .text                                    0x0800019c   Section       56  startup_stm32f10x_md.o(.text)
    .text                                    0x080001d4   Section        0  minibalance.o(.text)
    .text                                    0x08000318   Section        0  delay.o(.text)
    .text                                    0x080003c8   Section        0  sys.o(.text)
    .text                                    0x08000684   Section        0  usart.o(.text)
    .text                                    0x080007ac   Section        0  led.o(.text)
    .text                                    0x08000820   Section        0  key.o(.text)
    .text                                    0x08000a44   Section        0  oled.o(.text)
    .text                                    0x08000e88   Section        0  adc.o(.text)
    .text                                    0x080013bc   Section        0  timer.o(.text)
    .text                                    0x08001404   Section        0  motor.o(.text)
    .text                                    0x08001584   Section        0  encoder.o(.text)
    .text                                    0x080017d4   Section        0  usart3.o(.text)
    .text                                    0x08001ab0   Section        0  pstwo.o(.text)
    .text                                    0x08001ef0   Section        0  exti.o(.text)
    .text                                    0x08001f64   Section        0  stmflash.o(.text)
    .text                                    0x08002258   Section        0  control.o(.text)
    .text                                    0x08002cf8   Section        0  show.o(.text)
    .text                                    0x08003430   Section        0  datascope_dp.o(.text)
    .text                                    0x08003584   Section        2  use_no_semi_2.o(.text)
    .text                                    0x08003588   Section        0  noretval__2printf.o(.text)
    .text                                    0x080035a0   Section        0  __printf.o(.text)
    .text                                    0x08003608   Section        0  _printf_dec.o(.text)
    .text                                    0x0800367c   Section       68  rt_memclr.o(.text)
    .text                                    0x080036c0   Section        0  heapauxi.o(.text)
    .text                                    0x080036c6   Section        2  use_no_semi.o(.text)
    .text                                    0x080036c8   Section        0  _rserrno.o(.text)
    .text                                    0x080036de   Section        0  _printf_intcommon.o(.text)
    .text                                    0x08003790   Section        0  _printf_char_file.o(.text)
    .text                                    0x080037b4   Section       78  rt_memclr_w.o(.text)
    .text                                    0x08003804   Section        8  rt_errno_addr_intlibspace.o(.text)
    .text                                    0x0800380c   Section        0  _printf_char_common.o(.text)
    _printf_input_char                       0x0800380d   Thumb Code    10  _printf_char_common.o(.text)
    .text                                    0x0800383c   Section        0  ferror.o(.text)
    .text                                    0x08003844   Section        8  libspace.o(.text)
    .text                                    0x0800384c   Section       74  sys_stackheap_outer.o(.text)
    .text                                    0x08003896   Section        0  exit.o(.text)
    i.__ARM_fpclassify                       0x080038a2   Section        0  fpclassify.o(i.__ARM_fpclassify)
    i.__ieee754_rem_pio2                     0x080038cc   Section        0  rred.o(i.__ieee754_rem_pio2)
    i.__kernel_poly                          0x08003c54   Section        0  poly.o(i.__kernel_poly)
    i.__kernel_tan                           0x08003d00   Section        0  tan_i.o(i.__kernel_tan)
    i.__mathlib_dbl_underflow                0x08003f78   Section        0  dunder.o(i.__mathlib_dbl_underflow)
    i.pow                                    0x08003f88   Section        0  pow.o(i.pow)
    i.sqrt                                   0x08004968   Section        0  sqrt.o(i.sqrt)
    i.tan                                    0x080049b4   Section        0  tan.o(i.tan)
    x$fpl$d2f                                0x08004a28   Section       98  d2f.o(x$fpl$d2f)
    x$fpl$dadd                               0x08004a8c   Section      336  daddsub_clz.o(x$fpl$dadd)
    _dadd1                                   0x08004a9d   Thumb Code     0  daddsub_clz.o(x$fpl$dadd)
    x$fpl$dcheck1                            0x08004bdc   Section       16  dcheck1.o(x$fpl$dcheck1)
    x$fpl$dcmpinf                            0x08004bec   Section       24  dcmpi.o(x$fpl$dcmpinf)
    x$fpl$ddiv                               0x08004c04   Section      688  ddiv.o(x$fpl$ddiv)
    ddiv_entry                               0x08004c0b   Thumb Code     0  ddiv.o(x$fpl$ddiv)
    x$fpl$dfix                               0x08004eb4   Section       94  dfix.o(x$fpl$dfix)
    x$fpl$dflt                               0x08004f12   Section       46  dflt_clz.o(x$fpl$dflt)
    x$fpl$dfltu                              0x08004f40   Section       38  dflt_clz.o(x$fpl$dfltu)
    x$fpl$dleqf                              0x08004f68   Section      120  dleqf.o(x$fpl$dleqf)
    x$fpl$dmul                               0x08004fe0   Section      340  dmul.o(x$fpl$dmul)
    x$fpl$dnaninf                            0x08005134   Section      156  dnaninf.o(x$fpl$dnaninf)
    x$fpl$dretinf                            0x080051d0   Section       12  dretinf.o(x$fpl$dretinf)
    x$fpl$drleqf                             0x080051dc   Section      108  drleqf.o(x$fpl$drleqf)
    x$fpl$drsb                               0x08005248   Section       22  daddsub_clz.o(x$fpl$drsb)
    x$fpl$dsqrt                              0x08005260   Section      460  dsqrt_noumaal.o(x$fpl$dsqrt)
    x$fpl$dsub                               0x0800542c   Section      468  daddsub_clz.o(x$fpl$dsub)
    _dsub1                                   0x0800543d   Thumb Code     0  daddsub_clz.o(x$fpl$dsub)
    x$fpl$f2d                                0x08005600   Section       86  f2d.o(x$fpl$f2d)
    x$fpl$fadd                               0x08005658   Section      196  faddsub_clz.o(x$fpl$fadd)
    _fadd1                                   0x08005667   Thumb Code     0  faddsub_clz.o(x$fpl$fadd)
    x$fpl$fcmpinf                            0x0800571c   Section       24  fcmpi.o(x$fpl$fcmpinf)
    x$fpl$fdiv                               0x08005734   Section      388  fdiv.o(x$fpl$fdiv)
    _fdiv1                                   0x08005735   Thumb Code     0  fdiv.o(x$fpl$fdiv)
    x$fpl$ffix                               0x080058b8   Section       54  ffix.o(x$fpl$ffix)
    x$fpl$ffixu                              0x080058f0   Section       62  ffixu.o(x$fpl$ffixu)
    x$fpl$fflt                               0x08005930   Section       48  fflt_clz.o(x$fpl$fflt)
    x$fpl$ffltu                              0x08005960   Section       38  fflt_clz.o(x$fpl$ffltu)
    x$fpl$fleqf                              0x08005988   Section      104  fleqf.o(x$fpl$fleqf)
    x$fpl$fmul                               0x080059f0   Section      258  fmul.o(x$fpl$fmul)
    x$fpl$fnaninf                            0x08005af2   Section      140  fnaninf.o(x$fpl$fnaninf)
    x$fpl$fretinf                            0x08005b7e   Section       10  fretinf.o(x$fpl$fretinf)
    x$fpl$frleqf                             0x08005b88   Section       98  frleqf.o(x$fpl$frleqf)
    x$fpl$frsb                               0x08005bea   Section       20  faddsub_clz.o(x$fpl$frsb)
    x$fpl$fsub                               0x08005c00   Section      234  faddsub_clz.o(x$fpl$fsub)
    _fsub1                                   0x08005c0f   Thumb Code     0  faddsub_clz.o(x$fpl$fsub)
    x$fpl$retnan                             0x08005cea   Section      100  retnan.o(x$fpl$retnan)
    x$fpl$scalbn                             0x08005d4e   Section       92  scalbn.o(x$fpl$scalbn)
    x$fpl$trapveneer                         0x08005daa   Section       48  trapv.o(x$fpl$trapveneer)
    .constdata                               0x08005dda   Section     2660  oled.o(.constdata)
    x$fpl$usenofp                            0x08005dda   Section        0  usenofp.o(x$fpl$usenofp)
    .constdata                               0x08006840   Section      136  pow.o(.constdata)
    bp                                       0x08006840   Data          16  pow.o(.constdata)
    dp_h                                     0x08006850   Data          16  pow.o(.constdata)
    dp_l                                     0x08006860   Data          16  pow.o(.constdata)
    L                                        0x08006870   Data          48  pow.o(.constdata)
    P                                        0x080068a0   Data          40  pow.o(.constdata)
    .constdata                               0x080068c8   Section        8  qnan.o(.constdata)
    .constdata                               0x080068d0   Section      200  rred.o(.constdata)
    pio2s                                    0x080068d0   Data          48  rred.o(.constdata)
    twooverpi                                0x08006900   Data         152  rred.o(.constdata)
    .constdata                               0x08006998   Section       96  tan_i.o(.constdata)
    Todd                                     0x08006998   Data          48  tan_i.o(.constdata)
    Teven                                    0x080069c8   Data          48  tan_i.o(.constdata)
    .data                                    0x20000000   Section      124  minibalance.o(.data)
    .data                                    0x2000007c   Section        4  delay.o(.data)
    fac_us                                   0x2000007c   Data           1  delay.o(.data)
    fac_ms                                   0x2000007e   Data           2  delay.o(.data)
    .data                                    0x20000080   Section        4  usart.o(.data)
    .data                                    0x20000084   Section        4  led.o(.data)
    temp                                     0x20000084   Data           4  led.o(.data)
    .data                                    0x20000088   Section       15  key.o(.data)
    flag_key                                 0x20000088   Data           1  key.o(.data)
    count_key                                0x20000089   Data           1  key.o(.data)
    double_key                               0x2000008a   Data           1  key.o(.data)
    count_single                             0x2000008c   Data           2  key.o(.data)
    Forever_count                            0x2000008e   Data           2  key.o(.data)
    flag_key                                 0x20000090   Data           1  key.o(.data)
    Long_Press_count                         0x20000092   Data           2  key.o(.data)
    Long_Press                               0x20000094   Data           2  key.o(.data)
    flag                                     0x20000096   Data           1  key.o(.data)
    .data                                    0x20000098   Section        8  usart3.o(.data)
    Flag_PID                                 0x20000099   Data           1  usart3.o(.data)
    i                                        0x2000009a   Data           1  usart3.o(.data)
    j                                        0x2000009b   Data           1  usart3.o(.data)
    Data                                     0x2000009c   Data           4  usart3.o(.data)
    .data                                    0x200000a0   Section       36  pstwo.o(.data)
    .data                                    0x200000c4   Section       66  control.o(.data)
    Bias                                     0x200000d8   Data           4  control.o(.data)
    Pwm                                      0x200000dc   Data           4  control.o(.data)
    Last_bias                                0x200000e0   Data           4  control.o(.data)
    Bias                                     0x200000e4   Data           4  control.o(.data)
    Pwm                                      0x200000e8   Data           4  control.o(.data)
    Last_bias                                0x200000ec   Data           4  control.o(.data)
    Bias                                     0x200000f0   Data           4  control.o(.data)
    Last_Bias                                0x200000f4   Data           4  control.o(.data)
    i                                        0x200000f8   Data           2  control.o(.data)
    j                                        0x200000fa   Data           2  control.o(.data)
    Left                                     0x200000fc   Data           2  control.o(.data)
    Right                                    0x200000fe   Data           2  control.o(.data)
    Last_CCD_Zhongzhi                        0x20000100   Data           2  control.o(.data)
    value1_max                               0x20000102   Data           2  control.o(.data)
    value1_min                               0x20000104   Data           2  control.o(.data)
    .data                                    0x20000108   Section        9  show.o(.data)
    flag                                     0x20000110   Data           1  show.o(.data)
    .bss                                     0x20000114   Section      296  minibalance.o(.bss)
    .bss                                     0x2000023c   Section     1024  oled.o(.bss)
    .bss                                     0x2000063c   Section       50  usart3.o(.bss)
    Receive                                  0x2000063c   Data          50  usart3.o(.bss)
    .bss                                     0x2000066e   Section        9  pstwo.o(.bss)
    .bss                                     0x20000678   Section     1024  stmflash.o(.bss)
    .bss                                     0x20000a78   Section       42  datascope_dp.o(.bss)
    .bss                                     0x20000aa4   Section       96  libspace.o(.bss)
    HEAP                                     0x20000b08   Section      512  startup_stm32f10x_md.o(HEAP)
    Heap_Mem                                 0x20000b08   Data         512  startup_stm32f10x_md.o(HEAP)
    STACK                                    0x20000d08   Section     1024  startup_stm32f10x_md.o(STACK)
    Stack_Mem                                0x20000d08   Data        1024  startup_stm32f10x_md.o(STACK)
    __initial_sp                             0x20001108   Data           0  startup_stm32f10x_md.o(STACK)

    Global Symbols

    Symbol Name                              Value     Ov Type        Size  Object(Section)

    BuildAttributes$$THM_ISAv4$P$D$K$B$S$PE$A:L22UL41UL21$X:L11$S22US41US21$IEEE1$IW$USESV6$~STKCKD$USESV7$~SHL$OTIME$ROPI$IEEEX$EBA8$UX$STANDARDLIB$REQ8$PRES8$EABIv2 0x00000000   Number         0  anon$$obj.o ABSOLUTE
    __ARM_use_no_argv                        0x00000000   Number         0  minibalance.o ABSOLUTE
    __ARM_exceptions_init                     - Undefined Weak Reference
    __alloca_initialize                       - Undefined Weak Reference
    __cpp_initialize__aeabi_                  - Undefined Weak Reference
    __cxa_finalize                            - Undefined Weak Reference
    __rt_locale                               - Undefined Weak Reference
    __sigvec_lookup                           - Undefined Weak Reference
    _atexit_init                              - Undefined Weak Reference
    _call_atexit_fns                          - Undefined Weak Reference
    _clock_init                               - Undefined Weak Reference
    _fp_trap_init                             - Undefined Weak Reference
    _fp_trap_shutdown                         - Undefined Weak Reference
    _get_lc_collate                           - Undefined Weak Reference
    _get_lc_ctype                             - Undefined Weak Reference
    _get_lc_monetary                          - Undefined Weak Reference
    _get_lc_numeric                           - Undefined Weak Reference
    _get_lc_time                              - Undefined Weak Reference
    _getenv_init                              - Undefined Weak Reference
    _handle_redirection                       - Undefined Weak Reference
    _init_alloc                               - Undefined Weak Reference
    _init_user_alloc                          - Undefined Weak Reference
    _initio                                   - Undefined Weak Reference
    _mutex_acquire                            - Undefined Weak Reference
    _mutex_release                            - Undefined Weak Reference
    _printf_post_padding                      - Undefined Weak Reference
    _printf_pre_padding                       - Undefined Weak Reference
    _printf_truncate_signed                   - Undefined Weak Reference
    _printf_truncate_unsigned                 - Undefined Weak Reference
    _rand_init                                - Undefined Weak Reference
    _signal_finish                            - Undefined Weak Reference
    _signal_init                              - Undefined Weak Reference
    _terminate_alloc                          - Undefined Weak Reference
    _terminate_user_alloc                     - Undefined Weak Reference
    _terminateio                              - Undefined Weak Reference
    __Vectors_Size                           0x000000ec   Number         0  startup_stm32f10x_md.o ABSOLUTE
    __Vectors                                0x08000000   Data           4  startup_stm32f10x_md.o(RESET)
    __Vectors_End                            0x080000ec   Data           0  startup_stm32f10x_md.o(RESET)
    __main                                   0x080000ed   Thumb Code     8  __main.o(!!!main)
    __scatterload                            0x080000f5   Thumb Code     0  __scatter.o(!!!scatter)
    __scatterload_rt2                        0x080000f5   Thumb Code    44  __scatter.o(!!!scatter)
    __scatterload_rt2_thumb_only             0x080000f5   Thumb Code     0  __scatter.o(!!!scatter)
    __scatterload_null                       0x08000103   Thumb Code     0  __scatter.o(!!!scatter)
    __scatterload_copy                       0x08000129   Thumb Code    26  __scatter_copy.o(!!handler_copy)
    __scatterload_zeroinit                   0x08000145   Thumb Code    28  __scatter_zi.o(!!handler_zi)
    _printf_d                                0x08000161   Thumb Code     0  _printf_d.o(.ARM.Collect$$_printf_percent$$00000009)
    _printf_percent                          0x08000161   Thumb Code     0  _printf_percent.o(.ARM.Collect$$_printf_percent$$00000000)
    _printf_percent_end                      0x08000167   Thumb Code     0  _printf_percent_end.o(.ARM.Collect$$_printf_percent$$00000017)
    __rt_lib_init                            0x0800016b   Thumb Code     0  libinit.o(.ARM.Collect$$libinit$$00000000)
    __rt_lib_init_alloca_1                   0x0800016d   Thumb Code     0  libinit2.o(.ARM.Collect$$libinit$$0000002C)
    __rt_lib_init_argv_1                     0x0800016d   Thumb Code     0  libinit2.o(.ARM.Collect$$libinit$$0000002A)
    __rt_lib_init_atexit_1                   0x0800016d   Thumb Code     0  libinit2.o(.ARM.Collect$$libinit$$00000019)
    __rt_lib_init_clock_1                    0x0800016d   Thumb Code     0  libinit2.o(.ARM.Collect$$libinit$$0000001F)
    __rt_lib_init_cpp_1                      0x0800016d   Thumb Code     0  libinit2.o(.ARM.Collect$$libinit$$00000030)
    __rt_lib_init_exceptions_1               0x0800016d   Thumb Code     0  libinit2.o(.ARM.Collect$$libinit$$0000002E)
    __rt_lib_init_fp_1                       0x0800016d   Thumb Code     0  libinit2.o(.ARM.Collect$$libinit$$00000002)
    __rt_lib_init_fp_trap_1                  0x0800016d   Thumb Code     0  libinit2.o(.ARM.Collect$$libinit$$0000001D)
    __rt_lib_init_getenv_1                   0x0800016d   Thumb Code     0  libinit2.o(.ARM.Collect$$libinit$$00000021)
    __rt_lib_init_heap_1                     0x0800016d   Thumb Code     0  libinit2.o(.ARM.Collect$$libinit$$00000008)
    __rt_lib_init_lc_collate_1               0x0800016d   Thumb Code     0  libinit2.o(.ARM.Collect$$libinit$$0000000F)
    __rt_lib_init_lc_ctype_1                 0x0800016d   Thumb Code     0  libinit2.o(.ARM.Collect$$libinit$$00000011)
    __rt_lib_init_lc_monetary_1              0x0800016d   Thumb Code     0  libinit2.o(.ARM.Collect$$libinit$$00000013)
    __rt_lib_init_lc_numeric_1               0x0800016d   Thumb Code     0  libinit2.o(.ARM.Collect$$libinit$$00000015)
    __rt_lib_init_lc_time_1                  0x0800016d   Thumb Code     0  libinit2.o(.ARM.Collect$$libinit$$00000017)
    __rt_lib_init_rand_1                     0x0800016d   Thumb Code     0  libinit2.o(.ARM.Collect$$libinit$$0000000C)
    __rt_lib_init_return                     0x0800016d   Thumb Code     0  libinit2.o(.ARM.Collect$$libinit$$00000031)
    __rt_lib_init_signal_1                   0x0800016d   Thumb Code     0  libinit2.o(.ARM.Collect$$libinit$$0000001B)
    __rt_lib_init_stdio_1                    0x0800016d   Thumb Code     0  libinit2.o(.ARM.Collect$$libinit$$00000023)
    __rt_lib_init_user_alloc_1               0x0800016d   Thumb Code     0  libinit2.o(.ARM.Collect$$libinit$$0000000A)
    __rt_lib_shutdown                        0x0800016f   Thumb Code     0  libshutdown.o(.ARM.Collect$$libshutdown$$00000000)
    __rt_lib_shutdown_fp_trap_1              0x08000171   Thumb Code     0  libshutdown2.o(.ARM.Collect$$libshutdown$$00000006)
    __rt_lib_shutdown_heap_1                 0x08000171   Thumb Code     0  libshutdown2.o(.ARM.Collect$$libshutdown$$0000000E)
    __rt_lib_shutdown_return                 0x08000171   Thumb Code     0  libshutdown2.o(.ARM.Collect$$libshutdown$$0000000F)
    __rt_lib_shutdown_signal_1               0x08000171   Thumb Code     0  libshutdown2.o(.ARM.Collect$$libshutdown$$00000009)
    __rt_lib_shutdown_stdio_1                0x08000171   Thumb Code     0  libshutdown2.o(.ARM.Collect$$libshutdown$$00000003)
    __rt_lib_shutdown_user_alloc_1           0x08000171   Thumb Code     0  libshutdown2.o(.ARM.Collect$$libshutdown$$0000000B)
    __rt_entry                               0x08000173   Thumb Code     0  rtentry.o(.ARM.Collect$$rtentry$$00000000)
    __rt_entry_presh_1                       0x08000173   Thumb Code     0  rtentry2.o(.ARM.Collect$$rtentry$$00000002)
    __rt_entry_sh                            0x08000173   Thumb Code     0  rtentry4.o(.ARM.Collect$$rtentry$$00000004)
    __rt_entry_li                            0x08000179   Thumb Code     0  rtentry2.o(.ARM.Collect$$rtentry$$0000000A)
    __rt_entry_postsh_1                      0x08000179   Thumb Code     0  rtentry2.o(.ARM.Collect$$rtentry$$00000009)
    __rt_entry_main                          0x0800017d   Thumb Code     0  rtentry2.o(.ARM.Collect$$rtentry$$0000000D)
    __rt_entry_postli_1                      0x0800017d   Thumb Code     0  rtentry2.o(.ARM.Collect$$rtentry$$0000000C)
    __rt_exit                                0x08000185   Thumb Code     0  rtexit.o(.ARM.Collect$$rtexit$$00000000)
    __rt_exit_ls                             0x08000187   Thumb Code     0  rtexit2.o(.ARM.Collect$$rtexit$$00000003)
    __rt_exit_prels_1                        0x08000187   Thumb Code     0  rtexit2.o(.ARM.Collect$$rtexit$$00000002)
    __rt_exit_exit                           0x0800018b   Thumb Code     0  rtexit2.o(.ARM.Collect$$rtexit$$00000004)
    WFI_SET                                  0x08000191   Thumb Code     2  sys.o(.emb_text)
    INTX_DISABLE                             0x08000193   Thumb Code     2  sys.o(.emb_text)
    INTX_ENABLE                              0x08000195   Thumb Code     2  sys.o(.emb_text)
    MSR_MSP                                  0x08000197   Thumb Code     6  sys.o(.emb_text)
    Reset_Handler                            0x0800019d   Thumb Code     4  startup_stm32f10x_md.o(.text)
    NMI_Handler                              0x080001a1   Thumb Code     2  startup_stm32f10x_md.o(.text)
    HardFault_Handler                        0x080001a3   Thumb Code     2  startup_stm32f10x_md.o(.text)
    MemManage_Handler                        0x080001a5   Thumb Code     2  startup_stm32f10x_md.o(.text)
    BusFault_Handler                         0x080001a7   Thumb Code     2  startup_stm32f10x_md.o(.text)
    UsageFault_Handler                       0x080001a9   Thumb Code     2  startup_stm32f10x_md.o(.text)
    SVC_Handler                              0x080001ab   Thumb Code     2  startup_stm32f10x_md.o(.text)
    DebugMon_Handler                         0x080001ad   Thumb Code     2  startup_stm32f10x_md.o(.text)
    PendSV_Handler                           0x080001af   Thumb Code     2  startup_stm32f10x_md.o(.text)
    SysTick_Handler                          0x080001b1   Thumb Code     2  startup_stm32f10x_md.o(.text)
    ADC1_2_IRQHandler                        0x080001b3   Thumb Code     0  startup_stm32f10x_md.o(.text)
    CAN1_RX1_IRQHandler                      0x080001b3   Thumb Code     0  startup_stm32f10x_md.o(.text)
    CAN1_SCE_IRQHandler                      0x080001b3   Thumb Code     0  startup_stm32f10x_md.o(.text)
    DMA1_Channel1_IRQHandler                 0x080001b3   Thumb Code     0  startup_stm32f10x_md.o(.text)
    DMA1_Channel2_IRQHandler                 0x080001b3   Thumb Code     0  startup_stm32f10x_md.o(.text)
    DMA1_Channel3_IRQHandler                 0x080001b3   Thumb Code     0  startup_stm32f10x_md.o(.text)
    DMA1_Channel4_IRQHandler                 0x080001b3   Thumb Code     0  startup_stm32f10x_md.o(.text)
    DMA1_Channel5_IRQHandler                 0x080001b3   Thumb Code     0  startup_stm32f10x_md.o(.text)
    DMA1_Channel6_IRQHandler                 0x080001b3   Thumb Code     0  startup_stm32f10x_md.o(.text)
    DMA1_Channel7_IRQHandler                 0x080001b3   Thumb Code     0  startup_stm32f10x_md.o(.text)
    EXTI15_10_IRQHandler                     0x080001b3   Thumb Code     0  startup_stm32f10x_md.o(.text)
    EXTI2_IRQHandler                         0x080001b3   Thumb Code     0  startup_stm32f10x_md.o(.text)
    EXTI3_IRQHandler                         0x080001b3   Thumb Code     0  startup_stm32f10x_md.o(.text)
    EXTI4_IRQHandler                         0x080001b3   Thumb Code     0  startup_stm32f10x_md.o(.text)
    FLASH_IRQHandler                         0x080001b3   Thumb Code     0  startup_stm32f10x_md.o(.text)
    I2C1_ER_IRQHandler                       0x080001b3   Thumb Code     0  startup_stm32f10x_md.o(.text)
    I2C1_EV_IRQHandler                       0x080001b3   Thumb Code     0  startup_stm32f10x_md.o(.text)
    I2C2_ER_IRQHandler                       0x080001b3   Thumb Code     0  startup_stm32f10x_md.o(.text)
    I2C2_EV_IRQHandler                       0x080001b3   Thumb Code     0  startup_stm32f10x_md.o(.text)
    PVD_IRQHandler                           0x080001b3   Thumb Code     0  startup_stm32f10x_md.o(.text)
    RCC_IRQHandler                           0x080001b3   Thumb Code     0  startup_stm32f10x_md.o(.text)
    RTCAlarm_IRQHandler                      0x080001b3   Thumb Code     0  startup_stm32f10x_md.o(.text)
    RTC_IRQHandler                           0x080001b3   Thumb Code     0  startup_stm32f10x_md.o(.text)
    SPI1_IRQHandler                          0x080001b3   Thumb Code     0  startup_stm32f10x_md.o(.text)
    SPI2_IRQHandler                          0x080001b3   Thumb Code     0  startup_stm32f10x_md.o(.text)
    TAMPER_IRQHandler                        0x080001b3   Thumb Code     0  startup_stm32f10x_md.o(.text)
    TIM1_BRK_IRQHandler                      0x080001b3   Thumb Code     0  startup_stm32f10x_md.o(.text)
    TIM1_CC_IRQHandler                       0x080001b3   Thumb Code     0  startup_stm32f10x_md.o(.text)
    TIM1_TRG_COM_IRQHandler                  0x080001b3   Thumb Code     0  startup_stm32f10x_md.o(.text)
    TIM1_UP_IRQHandler                       0x080001b3   Thumb Code     0  startup_stm32f10x_md.o(.text)
    TIM4_IRQHandler                          0x080001b3   Thumb Code     0  startup_stm32f10x_md.o(.text)
    USART1_IRQHandler                        0x080001b3   Thumb Code     0  startup_stm32f10x_md.o(.text)
    USART2_IRQHandler                        0x080001b3   Thumb Code     0  startup_stm32f10x_md.o(.text)
    USBWakeUp_IRQHandler                     0x080001b3   Thumb Code     0  startup_stm32f10x_md.o(.text)
    USB_HP_CAN1_TX_IRQHandler                0x080001b3   Thumb Code     0  startup_stm32f10x_md.o(.text)
    USB_LP_CAN1_RX0_IRQHandler               0x080001b3   Thumb Code     0  startup_stm32f10x_md.o(.text)
    WWDG_IRQHandler                          0x080001b3   Thumb Code     0  startup_stm32f10x_md.o(.text)
    __user_initial_stackheap                 0x080001b5   Thumb Code     0  startup_stm32f10x_md.o(.text)
    main                                     0x080001d5   Thumb Code   282  minibalance.o(.text)
    delay_init                               0x08000319   Thumb Code    56  delay.o(.text)
    delay_us                                 0x08000351   Thumb Code    56  delay.o(.text)
    delay_ms                                 0x08000389   Thumb Code    56  delay.o(.text)
    MY_NVIC_SetVectorTable                   0x080003c9   Thumb Code    12  sys.o(.text)
    MY_NVIC_PriorityGroupConfig              0x080003d5   Thumb Code    36  sys.o(.text)
    MY_NVIC_Init                             0x080003f9   Thumb Code   116  sys.o(.text)
    Ex_NVIC_Config                           0x0800046d   Thumb Code   146  sys.o(.text)
    MYRCC_DeInit                             0x080004ff   Thumb Code    90  sys.o(.text)
    Sys_Standby                              0x08000559   Thumb Code    68  sys.o(.text)
    Sys_Soft_Reset                           0x0800059d   Thumb Code    12  sys.o(.text)
    JTAG_Set                                 0x080005a9   Thumb Code    42  sys.o(.text)
    Stm32_Clock_Init                         0x080005d3   Thumb Code   134  sys.o(.text)
    _sys_exit                                0x08000685   Thumb Code     6  usart.o(.text)
    fputc                                    0x0800068b   Thumb Code    60  usart.o(.text)
    usart1_send                              0x080006c7   Thumb Code    22  usart.o(.text)
    uart_init                                0x080006dd   Thumb Code   182  usart.o(.text)
    LED_Init                                 0x080007ad   Thumb Code    52  led.o(.text)
    Led_Flash                                0x080007e1   Thumb Code    44  led.o(.text)
    KEY_Init                                 0x08000821   Thumb Code    52  key.o(.text)
    click_N_Double                           0x08000855   Thumb Code   184  key.o(.text)
    click                                    0x0800090d   Thumb Code    38  key.o(.text)
    Long_Press                               0x08000933   Thumb Code    72  key.o(.text)
    select                                   0x0800097b   Thumb Code   138  key.o(.text)
    OLED_WR_Byte                             0x08000a45   Thumb Code    78  oled.o(.text)
    OLED_Refresh_Gram                        0x08000a93   Thumb Code    70  oled.o(.text)
    OLED_Display_On                          0x08000ad9   Thumb Code    28  oled.o(.text)
    OLED_Display_Off                         0x08000af5   Thumb Code    28  oled.o(.text)
    OLED_Clear                               0x08000b11   Thumb Code    42  oled.o(.text)
    OLED_DrawPoint                           0x08000b3b   Thumb Code   100  oled.o(.text)
    OLED_ShowChar                            0x08000b9f   Thumb Code   158  oled.o(.text)
    oled_pow                                 0x08000c3d   Thumb Code    22  oled.o(.text)
    OLED_ShowNumber                          0x08000c53   Thumb Code   148  oled.o(.text)
    OLED_ShowString                          0x08000ce7   Thumb Code    68  oled.o(.text)
    OLED_Init                                0x08000d2b   Thumb Code   348  oled.o(.text)
    Dly_us                                   0x08000e89   Thumb Code    12  adc.o(.text)
    Get_Adc                                  0x08000e95   Thumb Code    64  adc.o(.text)
    RD_TSL                                   0x08000ed5   Thumb Code   120  adc.o(.text)
    Adc_Init                                 0x08000f4d   Thumb Code   286  adc.o(.text)
    Get_battery_volt                         0x0800106b   Thumb Code    78  adc.o(.text)
    CCD                                      0x080010b9   Thumb Code    70  adc.o(.text)
    ccd_Init                                 0x080010ff   Thumb Code   326  adc.o(.text)
    ele_Init                                 0x08001245   Thumb Code   362  adc.o(.text)
    Timer_Init                               0x080013bd   Thumb Code    68  timer.o(.text)
    Motor_PWM_Init                           0x08001405   Thumb Code   228  motor.o(.text)
    Servo_PWM_Init                           0x080014e9   Thumb Code   136  motor.o(.text)
    Encoder_Init_TIM2                        0x08001585   Thumb Code    92  encoder.o(.text)
    Encoder_Init_TIM3                        0x080015e1   Thumb Code   224  encoder.o(.text)
    Read_Encoder                             0x080016c1   Thumb Code    70  encoder.o(.text)
    TIM3_IRQHandler                          0x08001707   Thumb Code    24  encoder.o(.text)
    EXTI1_IRQHandler                         0x0800171f   Thumb Code    78  encoder.o(.text)
    EXTI0_IRQHandler                         0x0800176d   Thumb Code    74  encoder.o(.text)
    uart3_init                               0x080017d5   Thumb Code   228  usart3.o(.text)
    USART3_IRQHandler                        0x080018b9   Thumb Code   432  usart3.o(.text)
    PS2_Init                                 0x08001ab1   Thumb Code   100  pstwo.o(.text)
    PS2_Cmd                                  0x08001b15   Thumb Code   128  pstwo.o(.text)
    PS2_RedLight                             0x08001b95   Thumb Code    50  pstwo.o(.text)
    PS2_ReadData                             0x08001bc7   Thumb Code   166  pstwo.o(.text)
    PS2_ClearData                            0x08001c6d   Thumb Code    20  pstwo.o(.text)
    PS2_DataKey                              0x08001c81   Thumb Code    70  pstwo.o(.text)
    PS2_AnologData                           0x08001cc7   Thumb Code     8  pstwo.o(.text)
    PS2_Vibration                            0x08001ccf   Thumb Code    90  pstwo.o(.text)
    PS2_ShortPoll                            0x08001d29   Thumb Code    62  pstwo.o(.text)
    PS2_EnterConfing                         0x08001d67   Thumb Code    86  pstwo.o(.text)
    PS2_TurnOnAnalogMode                     0x08001dbd   Thumb Code    80  pstwo.o(.text)
    PS2_VibrationMode                        0x08001e0d   Thumb Code    62  pstwo.o(.text)
    PS2_ExitConfing                          0x08001e4b   Thumb Code   138  pstwo.o(.text)
    PS2_SetInit                              0x08001ed5   Thumb Code    28  pstwo.o(.text)
    EXTI_Init                                0x08001ef1   Thumb Code    76  exti.o(.text)
    EXTI9_5_IRQHandler                       0x08001f3d   Thumb Code    20  exti.o(.text)
    STMFLASH_Unlock                          0x08001f65   Thumb Code    12  stmflash.o(.text)
    STMFLASH_Lock                            0x08001f71   Thumb Code    14  stmflash.o(.text)
    STMFLASH_GetStatus                       0x08001f7f   Thumb Code    38  stmflash.o(.text)
    STMFLASH_WaitDone                        0x08001fa5   Thumb Code    42  stmflash.o(.text)
    STMFLASH_ErasePage                       0x08001fcf   Thumb Code    72  stmflash.o(.text)
    STMFLASH_WriteHalfWord                   0x08002017   Thumb Code    58  stmflash.o(.text)
    STMFLASH_ReadHalfWord                    0x08002051   Thumb Code     6  stmflash.o(.text)
    STMFLASH_Write_NoCheck                   0x08002057   Thumb Code    38  stmflash.o(.text)
    STMFLASH_Read                            0x0800207d   Thumb Code    34  stmflash.o(.text)
    STMFLASH_Write                           0x0800209f   Thumb Code   224  stmflash.o(.text)
    Test_Write                               0x0800217f   Thumb Code    16  stmflash.o(.text)
    Flash_Read                               0x0800218f   Thumb Code   110  stmflash.o(.text)
    Flash_Write                              0x080021fd   Thumb Code    44  stmflash.o(.text)
    Kinematic_Analysis                       0x08002259   Thumb Code   236  control.o(.text)
    Set_Pwm                                  0x08002345   Thumb Code   110  control.o(.text)
    Xianfu_Pwm                               0x080023b3   Thumb Code    98  control.o(.text)
    Incremental_PI_B                         0x08002415   Thumb Code   114  control.o(.text)
    Incremental_PI_A                         0x08002487   Thumb Code   114  control.o(.text)
    Turn_Off                                 0x080024f9   Thumb Code    24  control.o(.text)
    myabs                                    0x08002511   Thumb Code    14  control.o(.text)
    Get_RC                                   0x0800251f   Thumb Code   814  control.o(.text)
    Find_CCD_Zhongzhi                        0x0800284d   Thumb Code   490  control.o(.text)
    Key                                      0x08002a37   Thumb Code    56  control.o(.text)
    TIM2_IRQHandler                          0x08002a6f   Thumb Code   568  control.o(.text)
    OLED_DrawPoint_Shu                       0x08002cf9   Thumb Code    60  show.o(.text)
    OLED_Show_CCD                            0x08002d35   Thumb Code    46  show.o(.text)
    oled_show                                0x08002d63   Thumb Code   780  show.o(.text)
    APP_Show                                 0x0800306f   Thumb Code   496  show.o(.text)
    DataScope                                0x0800325f   Thumb Code   124  show.o(.text)
    oled_show_once                           0x080032db   Thumb Code   136  show.o(.text)
    Float2Byte                               0x08003431   Thumb Code    28  datascope_dp.o(.text)
    DataScope_Get_Channel_Data               0x0800344d   Thumb Code   158  datascope_dp.o(.text)
    DataScope_Data_Generate                  0x080034eb   Thumb Code   148  datascope_dp.o(.text)
    __use_no_semihosting                     0x08003585   Thumb Code     2  use_no_semi_2.o(.text)
    __2printf                                0x08003589   Thumb Code    20  noretval__2printf.o(.text)
    __printf                                 0x080035a1   Thumb Code   104  __printf.o(.text)
    _printf_int_dec                          0x08003609   Thumb Code   100  _printf_dec.o(.text)
    __aeabi_memclr                           0x0800367d   Thumb Code     0  rt_memclr.o(.text)
    __rt_memclr                              0x0800367d   Thumb Code    68  rt_memclr.o(.text)
    _memset                                  0x08003681   Thumb Code     0  rt_memclr.o(.text)
    __use_two_region_memory                  0x080036c1   Thumb Code     2  heapauxi.o(.text)
    __rt_heap_escrow$2region                 0x080036c3   Thumb Code     2  heapauxi.o(.text)
    __rt_heap_expand$2region                 0x080036c5   Thumb Code     2  heapauxi.o(.text)
    __I$use$semihosting                      0x080036c7   Thumb Code     0  use_no_semi.o(.text)
    __use_no_semihosting_swi                 0x080036c7   Thumb Code     2  use_no_semi.o(.text)
    __read_errno                             0x080036c9   Thumb Code    10  _rserrno.o(.text)
    __set_errno                              0x080036d3   Thumb Code    12  _rserrno.o(.text)
    _printf_int_common                       0x080036df   Thumb Code   178  _printf_intcommon.o(.text)
    _printf_char_file                        0x08003791   Thumb Code    32  _printf_char_file.o(.text)
    __aeabi_memclr4                          0x080037b5   Thumb Code     0  rt_memclr_w.o(.text)
    __aeabi_memclr8                          0x080037b5   Thumb Code     0  rt_memclr_w.o(.text)
    __rt_memclr_w                            0x080037b5   Thumb Code    78  rt_memclr_w.o(.text)
    _memset_w                                0x080037b9   Thumb Code     0  rt_memclr_w.o(.text)
    __aeabi_errno_addr                       0x08003805   Thumb Code     8  rt_errno_addr_intlibspace.o(.text)
    __errno$intlibspace                      0x08003805   Thumb Code     0  rt_errno_addr_intlibspace.o(.text)
    __rt_errno_addr$intlibspace              0x08003805   Thumb Code     0  rt_errno_addr_intlibspace.o(.text)
    _printf_char_common                      0x08003817   Thumb Code    32  _printf_char_common.o(.text)
    ferror                                   0x0800383d   Thumb Code     8  ferror.o(.text)
    __user_libspace                          0x08003845   Thumb Code     8  libspace.o(.text)
    __user_perproc_libspace                  0x08003845   Thumb Code     0  libspace.o(.text)
    __user_perthread_libspace                0x08003845   Thumb Code     0  libspace.o(.text)
    __user_setup_stackheap                   0x0800384d   Thumb Code    74  sys_stackheap_outer.o(.text)
    exit                                     0x08003897   Thumb Code    12  exit.o(.text)
    __ARM_fpclassify                         0x080038a3   Thumb Code    40  fpclassify.o(i.__ARM_fpclassify)
    __ieee754_rem_pio2                       0x080038cd   Thumb Code   830  rred.o(i.__ieee754_rem_pio2)
    __kernel_poly                            0x08003c55   Thumb Code   170  poly.o(i.__kernel_poly)
    __kernel_tan                             0x08003d01   Thumb Code   582  tan_i.o(i.__kernel_tan)
    __mathlib_dbl_underflow                  0x08003f79   Thumb Code    10  dunder.o(i.__mathlib_dbl_underflow)
    pow                                      0x08003f89   Thumb Code  2510  pow.o(i.pow)
    sqrt                                     0x08004969   Thumb Code    76  sqrt.o(i.sqrt)
    tan                                      0x080049b5   Thumb Code   106  tan.o(i.tan)
    __aeabi_d2f                              0x08004a29   Thumb Code     0  d2f.o(x$fpl$d2f)
    _d2f                                     0x08004a29   Thumb Code    98  d2f.o(x$fpl$d2f)
    __aeabi_dadd                             0x08004a8d   Thumb Code     0  daddsub_clz.o(x$fpl$dadd)
    _dadd                                    0x08004a8d   Thumb Code   332  daddsub_clz.o(x$fpl$dadd)
    __fpl_dcheck_NaN1                        0x08004bdd   Thumb Code    10  dcheck1.o(x$fpl$dcheck1)
    __fpl_dcmp_Inf                           0x08004bed   Thumb Code    24  dcmpi.o(x$fpl$dcmpinf)
    __aeabi_ddiv                             0x08004c05   Thumb Code     0  ddiv.o(x$fpl$ddiv)
    _ddiv                                    0x08004c05   Thumb Code   552  ddiv.o(x$fpl$ddiv)
    __aeabi_d2iz                             0x08004eb5   Thumb Code     0  dfix.o(x$fpl$dfix)
    _dfix                                    0x08004eb5   Thumb Code    94  dfix.o(x$fpl$dfix)
    __aeabi_i2d                              0x08004f13   Thumb Code     0  dflt_clz.o(x$fpl$dflt)
    _dflt                                    0x08004f13   Thumb Code    46  dflt_clz.o(x$fpl$dflt)
    __aeabi_ui2d                             0x08004f41   Thumb Code     0  dflt_clz.o(x$fpl$dfltu)
    _dfltu                                   0x08004f41   Thumb Code    38  dflt_clz.o(x$fpl$dfltu)
    __aeabi_cdcmple                          0x08004f69   Thumb Code     0  dleqf.o(x$fpl$dleqf)
    _dcmple                                  0x08004f69   Thumb Code   120  dleqf.o(x$fpl$dleqf)
    __fpl_dcmple_InfNaN                      0x08004fcb   Thumb Code     0  dleqf.o(x$fpl$dleqf)
    __aeabi_dmul                             0x08004fe1   Thumb Code     0  dmul.o(x$fpl$dmul)
    _dmul                                    0x08004fe1   Thumb Code   332  dmul.o(x$fpl$dmul)
    __fpl_dnaninf                            0x08005135   Thumb Code   156  dnaninf.o(x$fpl$dnaninf)
    __fpl_dretinf                            0x080051d1   Thumb Code    12  dretinf.o(x$fpl$dretinf)
    __aeabi_cdrcmple                         0x080051dd   Thumb Code     0  drleqf.o(x$fpl$drleqf)
    _drcmple                                 0x080051dd   Thumb Code   108  drleqf.o(x$fpl$drleqf)
    __aeabi_drsub                            0x08005249   Thumb Code     0  daddsub_clz.o(x$fpl$drsb)
    _drsb                                    0x08005249   Thumb Code    22  daddsub_clz.o(x$fpl$drsb)
    _dsqrt                                   0x08005261   Thumb Code   456  dsqrt_noumaal.o(x$fpl$dsqrt)
    __aeabi_dsub                             0x0800542d   Thumb Code     0  daddsub_clz.o(x$fpl$dsub)
    _dsub                                    0x0800542d   Thumb Code   464  daddsub_clz.o(x$fpl$dsub)
    __aeabi_f2d                              0x08005601   Thumb Code     0  f2d.o(x$fpl$f2d)
    _f2d                                     0x08005601   Thumb Code    86  f2d.o(x$fpl$f2d)
    __aeabi_fadd                             0x08005659   Thumb Code     0  faddsub_clz.o(x$fpl$fadd)
    _fadd                                    0x08005659   Thumb Code   196  faddsub_clz.o(x$fpl$fadd)
    __fpl_fcmp_Inf                           0x0800571d   Thumb Code    24  fcmpi.o(x$fpl$fcmpinf)
    __aeabi_fdiv                             0x08005735   Thumb Code     0  fdiv.o(x$fpl$fdiv)
    _fdiv                                    0x08005735   Thumb Code   384  fdiv.o(x$fpl$fdiv)
    __aeabi_f2iz                             0x080058b9   Thumb Code     0  ffix.o(x$fpl$ffix)
    _ffix                                    0x080058b9   Thumb Code    54  ffix.o(x$fpl$ffix)
    __aeabi_f2uiz                            0x080058f1   Thumb Code     0  ffixu.o(x$fpl$ffixu)
    _ffixu                                   0x080058f1   Thumb Code    62  ffixu.o(x$fpl$ffixu)
    __aeabi_i2f                              0x08005931   Thumb Code     0  fflt_clz.o(x$fpl$fflt)
    _fflt                                    0x08005931   Thumb Code    48  fflt_clz.o(x$fpl$fflt)
    __aeabi_ui2f                             0x08005961   Thumb Code     0  fflt_clz.o(x$fpl$ffltu)
    _ffltu                                   0x08005961   Thumb Code    38  fflt_clz.o(x$fpl$ffltu)
    __aeabi_cfcmple                          0x08005989   Thumb Code     0  fleqf.o(x$fpl$fleqf)
    _fcmple                                  0x08005989   Thumb Code   104  fleqf.o(x$fpl$fleqf)
    __fpl_fcmple_InfNaN                      0x080059db   Thumb Code     0  fleqf.o(x$fpl$fleqf)
    __aeabi_fmul                             0x080059f1   Thumb Code     0  fmul.o(x$fpl$fmul)
    _fmul                                    0x080059f1   Thumb Code   258  fmul.o(x$fpl$fmul)
    __fpl_fnaninf                            0x08005af3   Thumb Code   140  fnaninf.o(x$fpl$fnaninf)
    __fpl_fretinf                            0x08005b7f   Thumb Code    10  fretinf.o(x$fpl$fretinf)
    __aeabi_cfrcmple                         0x08005b89   Thumb Code     0  frleqf.o(x$fpl$frleqf)
    _frcmple                                 0x08005b89   Thumb Code    98  frleqf.o(x$fpl$frleqf)
    __aeabi_frsub                            0x08005beb   Thumb Code     0  faddsub_clz.o(x$fpl$frsb)
    _frsb                                    0x08005beb   Thumb Code    20  faddsub_clz.o(x$fpl$frsb)
    __aeabi_fsub                             0x08005c01   Thumb Code     0  faddsub_clz.o(x$fpl$fsub)
    _fsub                                    0x08005c01   Thumb Code   234  faddsub_clz.o(x$fpl$fsub)
    __fpl_return_NaN                         0x08005ceb   Thumb Code   100  retnan.o(x$fpl$retnan)
    __ARM_scalbn                             0x08005d4f   Thumb Code    92  scalbn.o(x$fpl$scalbn)
    __fpl_cmpreturn                          0x08005dab   Thumb Code    48  trapv.o(x$fpl$trapveneer)
    __I$use$fp                               0x08005dda   Number         0  usenofp.o(x$fpl$usenofp)
    oled_asc2_1206                           0x08005dda   Data        1140  oled.o(.constdata)
    oled_asc2_1608                           0x0800624e   Data        1520  oled.o(.constdata)
    __mathlib_zero                           0x080068c8   Data           8  qnan.o(.constdata)
    Region$$Table$$Base                      0x080069f8   Number         0  anon$$obj.o(Region$$Table)
    Region$$Table$$Limit                     0x08006a18   Number         0  anon$$obj.o(Region$$Table)
    Flag_Way                                 0x20000000   Data           1  minibalance.o(.data)
    Flag_Show                                0x20000001   Data           1  minibalance.o(.data)
    Flag_Stop                                0x20000002   Data           1  minibalance.o(.data)
    Flag_Next                                0x20000003   Data           1  minibalance.o(.data)
    Encoder_Left                             0x20000004   Data           4  minibalance.o(.data)
    Encoder_Right                            0x20000008   Data           4  minibalance.o(.data)
    Encoder_A_EXTI                           0x2000000c   Data           4  minibalance.o(.data)
    Flag_Direction                           0x20000010   Data           4  minibalance.o(.data)
    Encoder_Temp                             0x20000014   Data           4  minibalance.o(.data)
    Velocity                                 0x20000018   Data           4  minibalance.o(.data)
    Velocity_Set                             0x2000001c   Data           4  minibalance.o(.data)
    Angle                                    0x20000020   Data           4  minibalance.o(.data)
    Angle_Set                                0x20000024   Data           4  minibalance.o(.data)
    Motor_A                                  0x20000028   Data           4  minibalance.o(.data)
    Motor_B                                  0x2000002c   Data           4  minibalance.o(.data)
    Servo                                    0x20000030   Data           4  minibalance.o(.data)
    Target_A                                 0x20000034   Data           4  minibalance.o(.data)
    Target_B                                 0x20000038   Data           4  minibalance.o(.data)
    Voltage                                  0x2000003c   Data           4  minibalance.o(.data)
    Show_Data_Mb                             0x20000040   Data           4  minibalance.o(.data)
    delay_50                                 0x20000044   Data           1  minibalance.o(.data)
    delay_flag                               0x20000045   Data           1  minibalance.o(.data)
    Velocity_KP                              0x20000048   Data           4  minibalance.o(.data)
    Velocity_KI                              0x2000004c   Data           4  minibalance.o(.data)
    PS2_LX                                   0x20000050   Data           4  minibalance.o(.data)
    PS2_LY                                   0x20000054   Data           4  minibalance.o(.data)
    PS2_RX                                   0x20000058   Data           4  minibalance.o(.data)
    PS2_RY                                   0x2000005c   Data           4  minibalance.o(.data)
    PS2_KEY                                  0x20000060   Data           4  minibalance.o(.data)
    Bluetooth_Velocity                       0x20000064   Data           1  minibalance.o(.data)
    APP_RX                                   0x20000065   Data           1  minibalance.o(.data)
    CCD_Zhongzhi                             0x20000066   Data           1  minibalance.o(.data)
    CCD_Yuzhi                                0x20000067   Data           1  minibalance.o(.data)
    PID_Send                                 0x20000068   Data           1  minibalance.o(.data)
    Flash_Send                               0x20000069   Data           1  minibalance.o(.data)
    Sensor_Left                              0x2000006c   Data           4  minibalance.o(.data)
    Sensor_Middle                            0x20000070   Data           4  minibalance.o(.data)
    Sensor_Right                             0x20000074   Data           4  minibalance.o(.data)
    Sensor                                   0x20000078   Data           4  minibalance.o(.data)
    __stdout                                 0x20000080   Data           4  usart.o(.data)
    Usart3_Receive                           0x20000098   Data           1  usart3.o(.data)
    Handkey                                  0x200000a0   Data           2  pstwo.o(.data)
    Comd                                     0x200000a2   Data           2  pstwo.o(.data)
    MASK                                     0x200000a4   Data          32  pstwo.o(.data)
    Flag_Target                              0x200000c4   Data           1  control.o(.data)
    Voltage_Temp                             0x200000c8   Data           4  control.o(.data)
    Voltage_Count                            0x200000cc   Data           4  control.o(.data)
    Voltage_All                              0x200000d0   Data           4  control.o(.data)
    sum                                      0x200000d4   Data           4  control.o(.data)
    i                                        0x20000108   Data           1  show.o(.data)
    Send_Count                               0x20000109   Data           1  show.o(.data)
    Vol                                      0x2000010c   Data           4  show.o(.data)
    ADV                                      0x20000114   Data         256  minibalance.o(.bss)
    PID_Parameter                            0x20000214   Data          20  minibalance.o(.bss)
    Flash_Parameter                          0x20000228   Data          20  minibalance.o(.bss)
    OLED_GRAM                                0x2000023c   Data        1024  oled.o(.bss)
    Data                                     0x2000066e   Data           9  pstwo.o(.bss)
    STMFLASH_BUF                             0x20000678   Data        1024  stmflash.o(.bss)
    DataScope_OutPut_Buffer                  0x20000a78   Data          42  datascope_dp.o(.bss)
    __libspace_start                         0x20000aa4   Data          96  libspace.o(.bss)
    __temporary_stack_top$libspace           0x20000b04   Data           0  libspace.o(.bss)



==============================================================================

Memory Map of the image

  Image Entry point : 0x080000ed

  Load Region LR_IROM1 (Base: 0x08000000, Size: 0x00006b2c, Max: 0x00010000, ABSOLUTE)

    Execution Region ER_IROM1 (Base: 0x08000000, Size: 0x00006a18, Max: 0x00010000, ABSOLUTE)

    Base Addr    Size         Type   Attr      Idx    E Section Name        Object

    0x08000000   0x000000ec   Data   RO            3    RESET               startup_stm32f10x_md.o
    0x080000ec   0x00000008   Code   RO          415  * !!!main             c_w.l(__main.o)
    0x080000f4   0x00000034   Code   RO          716    !!!scatter          c_w.l(__scatter.o)
    0x08000128   0x0000001a   Code   RO          718    !!handler_copy      c_w.l(__scatter_copy.o)
    0x08000142   0x00000002   PAD
    0x08000144   0x0000001c   Code   RO          720    !!handler_zi        c_w.l(__scatter_zi.o)
    0x08000160   0x00000000   Code   RO          410    .ARM.Collect$$_printf_percent$$00000000  c_w.l(_printf_percent.o)
    0x08000160   0x00000006   Code   RO          409    .ARM.Collect$$_printf_percent$$00000009  c_w.l(_printf_d.o)
    0x08000166   0x00000004   Code   RO          500    .ARM.Collect$$_printf_percent$$00000017  c_w.l(_printf_percent_end.o)
    0x0800016a   0x00000002   Code   RO          590    .ARM.Collect$$libinit$$00000000  c_w.l(libinit.o)
    0x0800016c   0x00000000   Code   RO          598    .ARM.Collect$$libinit$$00000002  c_w.l(libinit2.o)
    0x0800016c   0x00000000   Code   RO          601    .ARM.Collect$$libinit$$00000008  c_w.l(libinit2.o)
    0x0800016c   0x00000000   Code   RO          603    .ARM.Collect$$libinit$$0000000A  c_w.l(libinit2.o)
    0x0800016c   0x00000000   Code   RO          605    .ARM.Collect$$libinit$$0000000C  c_w.l(libinit2.o)
    0x0800016c   0x00000000   Code   RO          608    .ARM.Collect$$libinit$$0000000F  c_w.l(libinit2.o)
    0x0800016c   0x00000000   Code   RO          610    .ARM.Collect$$libinit$$00000011  c_w.l(libinit2.o)
    0x0800016c   0x00000000   Code   RO          612    .ARM.Collect$$libinit$$00000013  c_w.l(libinit2.o)
    0x0800016c   0x00000000   Code   RO          614    .ARM.Collect$$libinit$$00000015  c_w.l(libinit2.o)
    0x0800016c   0x00000000   Code   RO          616    .ARM.Collect$$libinit$$00000017  c_w.l(libinit2.o)
    0x0800016c   0x00000000   Code   RO          618    .ARM.Collect$$libinit$$00000019  c_w.l(libinit2.o)
    0x0800016c   0x00000000   Code   RO          620    .ARM.Collect$$libinit$$0000001B  c_w.l(libinit2.o)
    0x0800016c   0x00000000   Code   RO          622    .ARM.Collect$$libinit$$0000001D  c_w.l(libinit2.o)
    0x0800016c   0x00000000   Code   RO          624    .ARM.Collect$$libinit$$0000001F  c_w.l(libinit2.o)
    0x0800016c   0x00000000   Code   RO          626    .ARM.Collect$$libinit$$00000021  c_w.l(libinit2.o)
    0x0800016c   0x00000000   Code   RO          628    .ARM.Collect$$libinit$$00000023  c_w.l(libinit2.o)
    0x0800016c   0x00000000   Code   RO          632    .ARM.Collect$$libinit$$0000002A  c_w.l(libinit2.o)
    0x0800016c   0x00000000   Code   RO          634    .ARM.Collect$$libinit$$0000002C  c_w.l(libinit2.o)
    0x0800016c   0x00000000   Code   RO          636    .ARM.Collect$$libinit$$0000002E  c_w.l(libinit2.o)
    0x0800016c   0x00000000   Code   RO          638    .ARM.Collect$$libinit$$00000030  c_w.l(libinit2.o)
    0x0800016c   0x00000002   Code   RO          639    .ARM.Collect$$libinit$$00000031  c_w.l(libinit2.o)
    0x0800016e   0x00000002   Code   RO          659    .ARM.Collect$$libshutdown$$00000000  c_w.l(libshutdown.o)
    0x08000170   0x00000000   Code   RO          670    .ARM.Collect$$libshutdown$$00000003  c_w.l(libshutdown2.o)
    0x08000170   0x00000000   Code   RO          673    .ARM.Collect$$libshutdown$$00000006  c_w.l(libshutdown2.o)
    0x08000170   0x00000000   Code   RO          676    .ARM.Collect$$libshutdown$$00000009  c_w.l(libshutdown2.o)
    0x08000170   0x00000000   Code   RO          678    .ARM.Collect$$libshutdown$$0000000B  c_w.l(libshutdown2.o)
    0x08000170   0x00000000   Code   RO          681    .ARM.Collect$$libshutdown$$0000000E  c_w.l(libshutdown2.o)
    0x08000170   0x00000002   Code   RO          682    .ARM.Collect$$libshutdown$$0000000F  c_w.l(libshutdown2.o)
    0x08000172   0x00000000   Code   RO          493    .ARM.Collect$$rtentry$$00000000  c_w.l(rtentry.o)
    0x08000172   0x00000000   Code   RO          545    .ARM.Collect$$rtentry$$00000002  c_w.l(rtentry2.o)
    0x08000172   0x00000006   Code   RO          557    .ARM.Collect$$rtentry$$00000004  c_w.l(rtentry4.o)
    0x08000178   0x00000000   Code   RO          547    .ARM.Collect$$rtentry$$00000009  c_w.l(rtentry2.o)
    0x08000178   0x00000004   Code   RO          548    .ARM.Collect$$rtentry$$0000000A  c_w.l(rtentry2.o)
    0x0800017c   0x00000000   Code   RO          550    .ARM.Collect$$rtentry$$0000000C  c_w.l(rtentry2.o)
    0x0800017c   0x00000008   Code   RO          551    .ARM.Collect$$rtentry$$0000000D  c_w.l(rtentry2.o)
    0x08000184   0x00000002   Code   RO          595    .ARM.Collect$$rtexit$$00000000  c_w.l(rtexit.o)
    0x08000186   0x00000000   Code   RO          643    .ARM.Collect$$rtexit$$00000002  c_w.l(rtexit2.o)
    0x08000186   0x00000004   Code   RO          644    .ARM.Collect$$rtexit$$00000003  c_w.l(rtexit2.o)
    0x0800018a   0x00000006   Code   RO          645    .ARM.Collect$$rtexit$$00000004  c_w.l(rtexit2.o)
    0x08000190   0x0000000c   Code   RO          124    .emb_text           sys.o
    0x0800019c   0x00000038   Code   RO            4    .text               startup_stm32f10x_md.o
    0x080001d4   0x00000144   Code   RO           10    .text               minibalance.o
    0x08000318   0x000000b0   Code   RO          106    .text               delay.o
    0x080003c8   0x000002bc   Code   RO          125    .text               sys.o
    0x08000684   0x00000128   Code   RO          140    .text               usart.o
    0x080007ac   0x00000074   Code   RO          165    .text               led.o
    0x08000820   0x00000224   Code   RO          178    .text               key.o
    0x08000a44   0x00000442   Code   RO          191    .text               oled.o
    0x08000e86   0x00000002   PAD
    0x08000e88   0x00000534   Code   RO          210    .text               adc.o
    0x080013bc   0x00000048   Code   RO          222    .text               timer.o
    0x08001404   0x00000180   Code   RO          234    .text               motor.o
    0x08001584   0x00000250   Code   RO          246    .text               encoder.o
    0x080017d4   0x000002dc   Code   RO          258    .text               usart3.o
    0x08001ab0   0x00000440   Code   RO          277    .text               pstwo.o
    0x08001ef0   0x00000074   Code   RO          296    .text               exti.o
    0x08001f64   0x000002f4   Code   RO          311    .text               stmflash.o
    0x08002258   0x00000aa0   Code   RO          326    .text               control.o
    0x08002cf8   0x00000738   Code   RO          344    .text               show.o
    0x08003430   0x00000154   Code   RO          359    .text               datascope_dp.o
    0x08003584   0x00000002   Code   RO          379    .text               c_w.l(use_no_semi_2.o)
    0x08003586   0x00000002   PAD
    0x08003588   0x00000018   Code   RO          383    .text               c_w.l(noretval__2printf.o)
    0x080035a0   0x00000068   Code   RO          385    .text               c_w.l(__printf.o)
    0x08003608   0x00000074   Code   RO          387    .text               c_w.l(_printf_dec.o)
    0x0800367c   0x00000044   Code   RO          411    .text               c_w.l(rt_memclr.o)
    0x080036c0   0x00000006   Code   RO          413    .text               c_w.l(heapauxi.o)
    0x080036c6   0x00000002   Code   RO          491    .text               c_w.l(use_no_semi.o)
    0x080036c8   0x00000016   Code   RO          494    .text               c_w.l(_rserrno.o)
    0x080036de   0x000000b2   Code   RO          496    .text               c_w.l(_printf_intcommon.o)
    0x08003790   0x00000024   Code   RO          498    .text               c_w.l(_printf_char_file.o)
    0x080037b4   0x0000004e   Code   RO          501    .text               c_w.l(rt_memclr_w.o)
    0x08003802   0x00000002   PAD
    0x08003804   0x00000008   Code   RO          562    .text               c_w.l(rt_errno_addr_intlibspace.o)
    0x0800380c   0x00000030   Code   RO          564    .text               c_w.l(_printf_char_common.o)
    0x0800383c   0x00000008   Code   RO          566    .text               c_w.l(ferror.o)
    0x08003844   0x00000008   Code   RO          576    .text               c_w.l(libspace.o)
    0x0800384c   0x0000004a   Code   RO          579    .text               c_w.l(sys_stackheap_outer.o)
    0x08003896   0x0000000c   Code   RO          583    .text               c_w.l(exit.o)
    0x080038a2   0x00000028   Code   RO          520    i.__ARM_fpclassify  m_ws.l(fpclassify.o)
    0x080038ca   0x00000002   PAD
    0x080038cc   0x00000388   Code   RO          525    i.__ieee754_rem_pio2  m_ws.l(rred.o)
    0x08003c54   0x000000aa   Code   RO          522    i.__kernel_poly     m_ws.l(poly.o)
    0x08003cfe   0x00000002   PAD
    0x08003d00   0x00000278   Code   RO          538    i.__kernel_tan      m_ws.l(tan_i.o)
    0x08003f78   0x00000010   Code   RO          518    i.__mathlib_dbl_underflow  m_ws.l(dunder.o)
    0x08003f88   0x000009e0   Code   RO          474    i.pow               m_ws.l(pow.o)
    0x08004968   0x0000004c   Code   RO          531    i.sqrt              m_ws.l(sqrt.o)
    0x080049b4   0x00000074   Code   RO          484    i.tan               m_ws.l(tan.o)
    0x08004a28   0x00000062   Code   RO          417    x$fpl$d2f           fz_ws.l(d2f.o)
    0x08004a8a   0x00000002   PAD
    0x08004a8c   0x00000150   Code   RO          419    x$fpl$dadd          fz_ws.l(daddsub_clz.o)
    0x08004bdc   0x00000010   Code   RO          570    x$fpl$dcheck1       fz_ws.l(dcheck1.o)
    0x08004bec   0x00000018   Code   RO          591    x$fpl$dcmpinf       fz_ws.l(dcmpi.o)
    0x08004c04   0x000002b0   Code   RO          426    x$fpl$ddiv          fz_ws.l(ddiv.o)
    0x08004eb4   0x0000005e   Code   RO          429    x$fpl$dfix          fz_ws.l(dfix.o)
    0x08004f12   0x0000002e   Code   RO          434    x$fpl$dflt          fz_ws.l(dflt_clz.o)
    0x08004f40   0x00000026   Code   RO          433    x$fpl$dfltu         fz_ws.l(dflt_clz.o)
    0x08004f66   0x00000002   PAD
    0x08004f68   0x00000078   Code   RO          572    x$fpl$dleqf         fz_ws.l(dleqf.o)
    0x08004fe0   0x00000154   Code   RO          439    x$fpl$dmul          fz_ws.l(dmul.o)
    0x08005134   0x0000009c   Code   RO          503    x$fpl$dnaninf       fz_ws.l(dnaninf.o)
    0x080051d0   0x0000000c   Code   RO          505    x$fpl$dretinf       fz_ws.l(dretinf.o)
    0x080051dc   0x0000006c   Code   RO          507    x$fpl$drleqf        fz_ws.l(drleqf.o)
    0x08005248   0x00000016   Code   RO          420    x$fpl$drsb          fz_ws.l(daddsub_clz.o)
    0x0800525e   0x00000002   PAD
    0x08005260   0x000001cc   Code   RO          574    x$fpl$dsqrt         fz_ws.l(dsqrt_noumaal.o)
    0x0800542c   0x000001d4   Code   RO          421    x$fpl$dsub          fz_ws.l(daddsub_clz.o)
    0x08005600   0x00000056   Code   RO          441    x$fpl$f2d           fz_ws.l(f2d.o)
    0x08005656   0x00000002   PAD
    0x08005658   0x000000c4   Code   RO          443    x$fpl$fadd          fz_ws.l(faddsub_clz.o)
    0x0800571c   0x00000018   Code   RO          509    x$fpl$fcmpinf       fz_ws.l(fcmpi.o)
    0x08005734   0x00000184   Code   RO          450    x$fpl$fdiv          fz_ws.l(fdiv.o)
    0x080058b8   0x00000036   Code   RO          453    x$fpl$ffix          fz_ws.l(ffix.o)
    0x080058ee   0x00000002   PAD
    0x080058f0   0x0000003e   Code   RO          457    x$fpl$ffixu         fz_ws.l(ffixu.o)
    0x0800592e   0x00000002   PAD
    0x08005930   0x00000030   Code   RO          462    x$fpl$fflt          fz_ws.l(fflt_clz.o)
    0x08005960   0x00000026   Code   RO          461    x$fpl$ffltu         fz_ws.l(fflt_clz.o)
    0x08005986   0x00000002   PAD
    0x08005988   0x00000068   Code   RO          467    x$fpl$fleqf         fz_ws.l(fleqf.o)
    0x080059f0   0x00000102   Code   RO          469    x$fpl$fmul          fz_ws.l(fmul.o)
    0x08005af2   0x0000008c   Code   RO          511    x$fpl$fnaninf       fz_ws.l(fnaninf.o)
    0x08005b7e   0x0000000a   Code   RO          513    x$fpl$fretinf       fz_ws.l(fretinf.o)
    0x08005b88   0x00000062   Code   RO          471    x$fpl$frleqf        fz_ws.l(frleqf.o)
    0x08005bea   0x00000014   Code   RO          444    x$fpl$frsb          fz_ws.l(faddsub_clz.o)
    0x08005bfe   0x00000002   PAD
    0x08005c00   0x000000ea   Code   RO          445    x$fpl$fsub          fz_ws.l(faddsub_clz.o)
    0x08005cea   0x00000064   Code   RO          593    x$fpl$retnan        fz_ws.l(retnan.o)
    0x08005d4e   0x0000005c   Code   RO          515    x$fpl$scalbn        fz_ws.l(scalbn.o)
    0x08005daa   0x00000030   Code   RO          640    x$fpl$trapveneer    fz_ws.l(trapv.o)
    0x08005dda   0x00000000   Code   RO          517    x$fpl$usenofp       fz_ws.l(usenofp.o)
    0x08005dda   0x00000a64   Data   RO          193    .constdata          oled.o
    0x0800683e   0x00000002   PAD
    0x08006840   0x00000088   Data   RO          475    .constdata          m_ws.l(pow.o)
    0x080068c8   0x00000008   Data   RO          524    .constdata          m_ws.l(qnan.o)
    0x080068d0   0x000000c8   Data   RO          527    .constdata          m_ws.l(rred.o)
    0x08006998   0x00000060   Data   RO          539    .constdata          m_ws.l(tan_i.o)
    0x080069f8   0x00000020   Data   RO          714    Region$$Table       anon$$obj.o


    Execution Region RW_IRAM1 (Base: 0x20000000, Size: 0x00001108, Max: 0x00005000, ABSOLUTE)

    Base Addr    Size         Type   Attr      Idx    E Section Name        Object

    0x20000000   0x0000007c   Data   RW           12    .data               minibalance.o
    0x2000007c   0x00000004   Data   RW          107    .data               delay.o
    0x20000080   0x00000004   Data   RW          141    .data               usart.o
    0x20000084   0x00000004   Data   RW          166    .data               led.o
    0x20000088   0x0000000f   Data   RW          179    .data               key.o
    0x20000097   0x00000001   PAD
    0x20000098   0x00000008   Data   RW          260    .data               usart3.o
    0x200000a0   0x00000024   Data   RW          279    .data               pstwo.o
    0x200000c4   0x00000042   Data   RW          327    .data               control.o
    0x20000106   0x00000002   PAD
    0x20000108   0x00000009   Data   RW          345    .data               show.o
    0x20000111   0x00000003   PAD
    0x20000114   0x00000128   Zero   RW           11    .bss                minibalance.o
    0x2000023c   0x00000400   Zero   RW          192    .bss                oled.o
    0x2000063c   0x00000032   Zero   RW          259    .bss                usart3.o
    0x2000066e   0x00000009   Zero   RW          278    .bss                pstwo.o
    0x20000677   0x00000001   PAD
    0x20000678   0x00000400   Zero   RW          312    .bss                stmflash.o
    0x20000a78   0x0000002a   Zero   RW          360    .bss                datascope_dp.o
    0x20000aa2   0x00000002   PAD
    0x20000aa4   0x00000060   Zero   RW          577    .bss                c_w.l(libspace.o)
    0x20000b04   0x00000004   PAD
    0x20000b08   0x00000200   Zero   RW            2    HEAP                startup_stm32f10x_md.o
    0x20000d08   0x00000400   Zero   RW            1    STACK               startup_stm32f10x_md.o


==============================================================================

Image component sizes


      Code (inc. data)   RO Data    RW Data    ZI Data      Debug   Object Name

      1332         62          0          0          0       2076   adc.o
      2720        342          0         66          0       4291   control.o
       340         30          0          0         42       2242   datascope_dp.o
       176          8          0          4          0       1195   delay.o
       592         30          0          0          0       1497   encoder.o
       116         20          0          0          0        747   exti.o
       548         64          0         15          0       1782   key.o
       116         20          0          4          0        729   led.o
       324         42          0        124        296     208942   minibalance.o
       384         20          0          0          0        884   motor.o
      1090         46       2660          0       1024       4731   oled.o
      1088         52          0         36          9       3931   pstwo.o
      1848        424          0          9          0       2438   show.o
        56         22        236          0       1536        832   startup_stm32f10x_md.o
       756         48          0          0       1024       4338   stmflash.o
       712         44          0          0          0       2859   sys.o
        72          4          0          0          0        633   timer.o
       296         26          0          4          0       3186   usart.o
       732         82          0          8         50       1556   usart3.o

    ----------------------------------------------------------------------
     13300       1386       2930        276       3984     248889   Object Totals
         0          0         32          0          0          0   (incl. Generated)
         2          0          2          6          3          0   (incl. Padding)

    ----------------------------------------------------------------------

      Code (inc. data)   RO Data    RW Data    ZI Data      Debug   Library Member Name

         8          0          0          0          0         68   __main.o
       104          0          0          0          0         84   __printf.o
        52          8          0          0          0          0   __scatter.o
        26          0          0          0          0          0   __scatter_copy.o
        28          0          0          0          0          0   __scatter_zi.o
        48          6          0          0          0         96   _printf_char_common.o
        36          4          0          0          0         80   _printf_char_file.o
         6          0          0          0          0          0   _printf_d.o
       116         16          0          0          0         92   _printf_dec.o
       178          0          0          0          0         88   _printf_intcommon.o
         0          0          0          0          0          0   _printf_percent.o
         4          0          0          0          0          0   _printf_percent_end.o
        22          0          0          0          0        100   _rserrno.o
        12          0          0          0          0         72   exit.o
         8          0          0          0          0         68   ferror.o
         6          0          0          0          0        152   heapauxi.o
         2          0          0          0          0          0   libinit.o
         2          0          0          0          0          0   libinit2.o
         2          0          0          0          0          0   libshutdown.o
         2          0          0          0          0          0   libshutdown2.o
         8          4          0          0         96         68   libspace.o
        24          4          0          0          0         84   noretval__2printf.o
         8          4          0          0          0         68   rt_errno_addr_intlibspace.o
        68          0          0          0          0         68   rt_memclr.o
        78          0          0          0          0         80   rt_memclr_w.o
         0          0          0          0          0          0   rtentry.o
        12          0          0          0          0          0   rtentry2.o
         6          0          0          0          0          0   rtentry4.o
         2          0          0          0          0          0   rtexit.o
        10          0          0          0          0          0   rtexit2.o
        74          0          0          0          0         80   sys_stackheap_outer.o
         2          0          0          0          0         68   use_no_semi.o
         2          0          0          0          0         68   use_no_semi_2.o
        98          4          0          0          0         92   d2f.o
       826         16          0          0          0        348   daddsub_clz.o
        16          4          0          0          0         68   dcheck1.o
        24          0          0          0          0         68   dcmpi.o
       688        140          0          0          0        208   ddiv.o
        94          4          0          0          0         92   dfix.o
        84          0          0          0          0        136   dflt_clz.o
       120          4          0          0          0         92   dleqf.o
       340         12          0          0          0        104   dmul.o
       156          4          0          0          0         92   dnaninf.o
        12          0          0          0          0         68   dretinf.o
       108          0          0          0          0         80   drleqf.o
       460         56          0          0          0        120   dsqrt_noumaal.o
        86          4          0          0          0         84   f2d.o
       450          8          0          0          0        236   faddsub_clz.o
        24          0          0          0          0         68   fcmpi.o
       388         76          0          0          0         96   fdiv.o
        54          4          0          0          0         84   ffix.o
        62          4          0          0          0         84   ffixu.o
        86          0          0          0          0        136   fflt_clz.o
       104          4          0          0          0         84   fleqf.o
       258          4          0          0          0         84   fmul.o
       140          4          0          0          0         84   fnaninf.o
        10          0          0          0          0         68   fretinf.o
        98          0          0          0          0         68   frleqf.o
       100          0          0          0          0         68   retnan.o
        92          0          0          0          0         68   scalbn.o
        48          0          0          0          0         68   trapv.o
         0          0          0          0          0          0   usenofp.o
        16          6          0          0          0         68   dunder.o
        40          0          0          0          0         68   fpclassify.o
       170          0          0          0          0         96   poly.o
      2528        190        136          0          0        332   pow.o
         0          0          8          0          0          0   qnan.o
       904         74        200          0          0        140   rred.o
        76          0          0          0          0         84   sqrt.o
       116         10          0          0          0        104   tan.o
       632         50         96          0          0        168   tan_i.o

    ----------------------------------------------------------------------
     10490        728        440          0        100       5492   Library Totals
        26          0          0          0          4          0   (incl. Padding)

    ----------------------------------------------------------------------

      Code (inc. data)   RO Data    RW Data    ZI Data      Debug   Library Name

       956         46          0          0         96       1484   c_w.l
      5026        352          0          0          0       2948   fz_ws.l
      4482        330        440          0          0       1060   m_ws.l

    ----------------------------------------------------------------------
     10490        728        440          0        100       5492   Library Totals

    ----------------------------------------------------------------------

==============================================================================


      Code (inc. data)   RO Data    RW Data    ZI Data      Debug   

     23790       2114       3370        276       4084     249853   Grand Totals
     23790       2114       3370        276       4084     249853   ELF Image Totals
     23790       2114       3370        276          0          0   ROM Totals

==============================================================================

    Total RO  Size (Code + RO Data)                27160 (  26.52kB)
    Total RW  Size (RW Data + ZI Data)              4360 (   4.26kB)
    Total ROM Size (Code + RO Data + RW Data)      27436 (  26.79kB)

==============================================================================

